:020000040800F2
:10000000981300209502000827260008D51600083E
:10001000252600081B160008192F00080000000004
:100020000000000000000000000000003D28000863
:100030001D160008000000001D28000851290008B6
:10004000AF020008AF020008AF020008AF020008CC
:10005000AF020008AF020008AF020008AF020008BC
:10006000AF020008AF020008AF020008AF020008AC
:10007000AF020008AF020008AF020008AF0200089C
:10008000AF020008AF020008AF020008AF0200088C
:10009000AF020008AF020008AF020008AF0200087C
:1000A000AF020008AF020008AF020008AF0200086C
:1000B000292A0008292D000800000000AF020008CE
:1000C000AF0200080000000000000000AF020008BE
:1000D00000000000AF020008AF020008AF020008F5
:1000E000AF020008AF02000800000000000000009E
:1000F0000000000000000000000000000000000000
:1001000000000000000000000000000000000000EF
:1001100000000000000000009D2D0008AF02000854
:1001200000000000000000000000000000000000CF
:1001300000000000000000000000000000000000BF
:10014000AF020008AF02000800000000000000003D
:10015000000000000000000000000000000000009F
:10016000000000000000000000000000000000008F
:10017000000000000000000000000000000000007F
:1001800000000000AF02000800F002F800F072F872
:100190000AA090E8000C82448344AAF10107DA45E2
:1001A00001D100F067F8AFF2090EBAE80F0013F0C2
:1001B000010F18BFFB1A43F0010318476CAE000093
:1001C0008CAE00000A444FF0000C10F8013B13F015
:1001D000070408BF10F8014B1D1108BF10F8015BA0
:1001E000641E05D010F8016B641E01F8016BF9D193
:1001F00013F0080F1EBF10F8014BAD1C0C1B09D1EA
:100200006D1E58BF01F801CBFAD505E014F8016B5B
:1002100001F8016B6D1EF9D59142D6D370470000ED
:100220000023002400250026103A28BF78C1FBD8FF
:10023000520728BF30C148BF0B607047662909F0DC
:100240003E81642900F0AA80782900F0E3807329B8
:1002500000F09D84002070471FB509F026F900F0DA
:100260009BFC04000020002108F0CAFAE0601FBDDA
:1002700010B510BD00F094FD1146FFF7EDFF05F03D
:1002800035F800F0B2FD03B4FFF7F2FF03BC00F055
:10029000F5FD00000948804709480047FEE7FEE7F2
:1002A000FEE7FEE7FEE7FEE7FEE7FEE7FEE7FEE726
:1002B00004480549054A064B70470000192A000802
:1002C00089010008980B002098130020980D002049
:1002D000980D00200FB41CB5074B06AA7B44694655
:1002E0000090059800F029FC0020694600F038FCD9
:1002F0001CBC5DF814FB00008108000070B50446CA
:1003000085690068C10601D5302600E02026C007B7
:1003100007D070BDD4E9012130469047206A401CC7
:1003200020626D1EF6D570BD70B5044685690078F3
:10033000C00707D170BDD4E9012120209047206A71
:10034000401C20626D1EF6D570BD70B50C4605468A
:10035000012A05D02878800600D5EA69002302E04A
:10036000012305E05B1C934202D2E05C0028F9D136
:10037000A869E618C01AA861286A184428622846A5
:10038000FFF7BCFF04E0D5E9012114F8010B904709
:10039000B442F8D32846FFF7C7FF70BD2DE9F041FE
:1003A0000646002410687529314616A510D0AFF313
:1003B0000080002802DA404213A507E031688A076E
:1003C00001D512A502E0490704D511A5012401E0D9
:1003D000AFF3008000210A2206F1240709E0B0FBF8
:1003E000F2FCB0FBF2F302FB1C00303078541846EC
:1003F000491C0028F3D123462A463046BDE8F04187
:1004000000F02DB9000000002D0000002B000000BE
:100410002000000070B504460D4621461068AFF379
:1004200000802188090502D50F4A7A4402E00E4A6D
:100430007A440E32002104F1240305E000F00F0697
:100440000009965D5E54491C0028F7D120780023EE
:10045000000704D5702D02D009B1022311322046C5
:10046000BDE8704000F0FBB866A500002DE9F05F24
:10047000894604464FF0000ADFF874B1FB44C0F827
:1004800020A02046E1688847002874D0252806D09F
:10049000D4E901219047206A401C2062F1E7002640
:1004A0005F462046E16888472028054607DB312D56
:1004B00005D2781910F8200C08B10643F1E7B0070F
:1004C00001D526F00406C4F81CA00027C4F818A023
:1004D0002A2D09D0284604F0B7F938B304EB870871
:1004E000303DC8F8185019E059F8041B204604EBB9
:1004F00087029161E1688847012F054618D1E069BC
:10050000002820DA26F020061DE0D8F8180000EBBD
:10051000800005EB40003038C8F818002046E1683C
:100520008847054604F090F90028EED1012F0AD043
:100530002E2D08D12046E16888477F1C0546022FF2
:1005400046F02006C4DBA069002803DA404246F0EA
:100550000106A061F00701D026F010066C2D0BD02B
:10056000682D09D04C2D39D06A2D35D0742D35D059
:100570007A2D33D016E038E0E1682F4620468847D0
:10058000B842054609D16C2F26D04FF48060E1684F
:10059000064320468847054604E06C2F1AD04FF4E6
:1005A000807006430DB3A5F14100192802D820350B
:1005B00046F400664A462946204626604E46FFF726
:1005C0003DFE80B101280BD0F61D26F0070000F19A
:1005D000080956E74020E4E78020D8E70020D6E766
:1005E00006F104094DE7284652E7206ABDE8F09F6E
:1005F0003CA500004FF0000200B513469446964615
:10060000203922BFA0E80C50A0E80C50B1F1200125
:10061000BFF4F7AF090728BFA0E80C5048BF0CC0D3
:100620005DF804EB890028BF40F8042B08BF704731
:1006300048BF20F8022B11F0804F18BF00F8012BA3
:10064000704770477047704710B500F0A9FA00680E
:1006500010BD10B5044600F0A3FA046010BD2DE9EA
:10066000F0470D4699469246044600F12408016879
:10067000880604D5E06921F01001216000E0012026
:10068000A84201DD471B00E00027A1697A1902EBAF
:100690000900081AA0612078C00602D42046FFF79E
:1006A0002DFE002608E0D4E901211AF80600904743
:1006B000206A401C761C20624E45F4DB2078C00680
:1006C0000AD52046FFF71AFE06E0D4E901213020C2
:1006D0009047206A401C2062381EA7F10107F4DC15
:1006E00007E0D4E9012118F805009047206A401C72
:1006F0002062281EA5F10105F3DC2046FFF714FE59
:100700002078000602D50220BDE8F0870120FBE733
:1007100070472DE9FF4F0C461E464FF0FF378BB058
:10072000D2E90001DDF860800A908A46C1F30A55DB
:1007300005B93D46002108464FF00000BAF1000F10
:1007400000F4400005DA00EB80004FF4400101EABC
:1007500050004FEA9059B9F1010F00DDB9460A98EF
:1007600050EA4A000ED044F61050A5F2FF3545433A
:100770002F14B8F1000F1ED07542291E1EDDC9F1DD
:1007800000021CE0B8F1010F4FF0000001D0302151
:1007900003E0F24305E02154401CB042FBDB30464D
:1007A0000022002121540B99C1F80880C1E90020E2
:1007B0000FB0BDE8F08FBD1B6D1CDEE74A4600DAC6
:1007C000694206A800F076FA06AB93E8070003AB8F
:1007D00083E8070050460A9900F057FB8DE80700B0
:1007E000A0F500501F3800900398002D0ADD42F25A
:1007F0001F014A460844002303A90390684600F0FD
:10080000C0FD09E0A0F500504A461F38002303A9A7
:100810000390684600F0CAFD8DE807000004000C54
:1008200003D04FF0FF30410800E01046B8F1000F50
:1008300003D00022009215461EE0751E05D400F07C
:10084000B3F9303262556D1EF9D5B3460122084323
:1008500002D000227F1C04E02078302801D1002241
:100860007F1E002A099784D01DE0112D07DA00F0C1
:100870009BF9303262556D1C50EA0102F5D10843F4
:1008800002D00098C8B10EE00021681E05E0235C8C
:10089000625C63542254401E491C8142F7DBAB4624
:1008A000A81B401E0990002004F80B000B98099A21
:1008B000C0F80880C0E9002B7AE711264FF0000845
:1008C00057E72DE9F04F88460446D21D22F0070174
:1008D00091B0D1E90001CDE90A0102F003FC024622
:1008E0000B98C00F01D02D2007E02068810701D5AB
:1008F0002B2002E0202101EAC000032A099001D048
:10090000072A05DB03464146204600F093F90BE138
:100910002078800601D5E06900E00620B8F1650F77
:10092000814606D0B8F1660F18D0B8F1670F70D1C4
:1009300031E00020B9F1110F009001DB112301E03B
:1009400009F101030AAA01A90CA8FFF7E2FEDDE9FB
:100950000C70002609F10105834647E001204B4653
:1009600000904FF000470AAA01A90CA8FFF7D1FE9A
:10097000DDE90DB00C995D46002610B909F10100C2
:100980000D18B9EB050003D4C0F1FF3609F10105DC
:10099000A5EB09002BE0B9F1010F01DA4FF00109D5
:1009A0000020B9F1110F0090484601DD112300E04D
:1009B00003460AAA01A90CA8FFF7ABFEDDE90C70FB
:1009C0004D4600268346207800070AD4AB4500DA5E
:1009D0005D4601A8012D04DD411911F8011C3029E3
:1009E00007D04F4502DA17F1040F04DA01208246DE
:1009F0000FE06D1EEEE7002F02DCED1B3E4403E02E
:100A0000781CA84200DD7D1CB81B00F1010A4FF0E4
:100A100000472078000703D4AA4501DB4FF0FF3AD6
:100A20000021B7F1004F0DF143088DF8431024D099
:100A300002202B23002F01DA7F422D230A21021EE0
:100A4000A0F1010000DC5FB197FBF1FC97FBF1F234
:100A500001FB1C7C17460CF1300C08F801CDEEE7C9
:100A6000A8F1010003702188090501D5452100E0A6
:100A70006521A0F1010800F8011C09980FA9A1EB5C
:100A80000807FF1D00B10120411901EBEA70A169BF
:100A90003844081A401EA0612078C00602D42046BF
:100AA000FFF72CFC099828B1D4E901219047206A6E
:100AB000401C20622078C00622D52046FFF71EFC8D
:100AC0001EE0002E04DBB34502DD01A8805D00E0DE
:100AD0003020D4E901219047206A401C2062761C16
:100AE000AAF101005FEA000A0AD100F055F8C068D7
:100AF0000168405CD4E901219047206A401C2062D3
:100B0000281EA5F10105DCDC07E0D4E9012118F875
:100B1000010B9047206A401C2062381EA7F1010794
:100B2000F3DC2046FFF700FC032011B041E6000093
:100B300001694A1C02610878704700B58FB0CDE9A1
:100B400001310021059105497944CDE90310114691
:100B50006846FFF78BFC0FB000BD0000E5FFFFFF0C
:100B60000A6802F8010B0A60704710B5436913B1B7
:100B7000AFF3008001E0FFF7E8FB012010BD127821
:100B800000F124010A7000224A700122EDE7116889
:100B90004FF0FF32E9E7000000487047580B002093
:100BA00000487047380B002030B5B0F10A024FEA18
:100BB000900E71F100034EEA817EB0EB0E0061EB06
:100BC00091014FEA101E4EEA017E10EB0E0041EB40
:100BD00011114FEA102E4EEA016E10EB0E0041EBA0
:100BE00011214FEA104E4EEA014E10EB0E0041EB80
:100BF0001141401841F100014FEAD00040EA417034
:100C00004FEAD10110EB80054FEA810444EA907469
:100C100044EB01046D1944EB0404521BA3414FF053
:100C2000000348BF0A3200D530BD401C41F100012D
:100C300030BD00002DE9F0411F460446032601683F
:100C4000072A01F4006004DB08B116A505E016A52B
:100C500003E008B115A500E015A521F01000206003
:100C6000A069C01EA0610FB1401EA0612046FFF721
:100C700045FB4FB1D4E9012138469047206A401C1A
:100C80002062C01C206206E0206AFAE7D4E9012154
:100C900015F8010B9047761EF8D22046FFF744FB6B
:100CA000BDE8F0814E414E006E616E00494E460037
:100CB000696E66002DE9F047814616468AB03548D0
:100CC00078440DC88DE80D0032487844801C03AC90
:100CD0000DC884E80D0041F69B300844372190FB95
:100CE000F1F290FBF1F5A5F1800501FB12041B3C2C
:100CF00002D56442012000E00020DFF898A0804681
:100D00000027FA44AAF1BE0A0EE0E0070AD03246F4
:100D1000684607EB470101230AEB810100F046FB1F
:100D20008DE8070064107F1C002CEED1194F7F4422
:100D3000AE3F19E0E80715D007EB04100DF1180AD3
:100D400090E80E008AE80E00C068F04201D19819C0
:100D500008903246012306A903A800F027FB03AB45
:100D600083E807006D10641C002DE3D14FF00103F0
:100D700032466946B8F1000F03A802D000F001FB2B
:100D800001E000F013FBC9E90001C9F808200AB02E
:100D9000BDE8F087E09F000000487047380B002056
:100DA0007546FFF7F9FFAE4605006946534620F049
:100DB0000700854618B020B5FFF77AFABDE8204055
:100DC0004FF000064FF000074FF000084FF0000B07
:100DD00021F00701AC46ACE8C009ACE8C009ACE8BA
:100DE000C009ACE8C0098D46704710B50446AFF3A2
:100DF00000802046BDE81040FFF745BA4FF0013CA7
:100E000050F8042B51F8043B9A4221D1A2EB0C0379
:100E1000934313EACC1317D150F8042B51F8043B39
:100E20009A4215D1A2EB0C03934313EACC130BD1D6
:100E300050F8042B51F8043B9A4209D1A2EB0C0361
:100E4000934313EACC13DBD04FF00000704700BF90
:100E5000D01A01BAB1FA81F101F0180122FA01F0B9
:100E6000CB40C1F12001DBB2C0B2C01A2CFA01F3B1
:100E7000D11A914311EAC311E6D1704701491820F4
:100E8000ABBEFEE72600020070475FEA400C08BFD9
:100E900091F0000F4FEA8C234FEAC12243EA5151EF
:100EA0004FEA1C5018BF00F5F0404FEA300018BF61
:100EB00041F000415FEA6C5C00F02980BCF1FF3F2B
:100EC00008BF40F080407047130C06BF12044FF07B
:100ED000100C4FF0000C130E04BF12020CF1080CA2
:100EE000130F04BF12010CF1040C930F04BF920006
:100EF0000CF1020CD30F04BF52000CF1010C11468F
:100F00004FF00002A0F11F00A0EB0C00704711F0A1
:100F1000004F08BF704731F000413FF4D5AF0B0CD4
:100F200006BF09044FF0100C4FF0000C0B0E04BF6D
:100F300009020CF1080C0B0F04BF09010CF1040CA1
:100F40008B0F04BF89000CF1020CCB0F04BF4900CA
:100F50000CF1010CCCF12003A0EB0C0022FA03F3FE
:100F600002FA0CF241EA030100F10100704720F09F
:100F70007F4C80EA030023F07F47ACEB070303F5C7
:100F80007C5300F0004003F1FF032DE980494FEA54
:100F9000154B09B44FEA144325EA0B4E24EA0348E3
:100FA0000FF2042606EB132749083E785FEA320267
:100FB00003FB0667C7F5000707FB06F64FEA543741
:100FC0004FEAD64606F1020607FB066CCCF1005C40
:100FD0004FEA1C472CEA074C07FB06F40CFB06F50E
:100FE00004EB15464FEA961634BF00204FF0004040
:100FF0004FEAD13706FB07FC4FEA1C4C0CFB0BF702
:10100000D21B03FB0CF761EB07010CFB0EF7B0EBF7
:10101000074072EB17420CFB08F734BFA2EB074204
:10102000B2EB074261EB17414FEA0C444FEA9107DC
:1010300006FB07FC4FEA1C4C0CFB0BF7B0EBC74060
:1010400072EB573203FB0CF734BFA2EBC742B2EB93
:10105000C74261EB57310CFB0EF7B0EBC70072EBE8
:1010600057720CFB08F734BFA2EBC702B2EBC70202
:1010700061EB5771039F4FEA816141EA921104EBE2
:10108000CC044FEAD1374FEA826206FB07FC42EA02
:1010900090124FEA80604FEA1C4C0CFB0BF7D21BFE
:1010A00003FB0CF761EB07010CFB0EF7B0EB0740FD
:1010B00072EB17420CFB08F734BFA2EB0742B2EB0E
:1010C000074261EB17414FEA8C554FEA910704EB59
:1010D0009C2406FB07FC4FEA1C4C0CFB0BF7B0EB07
:1010E000C74072EB573203FB0CF734BFA2EBC74289
:1010F000B2EBC74261EB57310CFB0EF7B0EBC70008
:1011000072EB57720CFB08F734BFA2EBC702B2EBCD
:10111000C70261EB577115EB4C254FEA816141EA3B
:1011200092114FEA82624FEAD13742EA901206FBEF
:1011300007FC44F100044FEA80604FEA1C4C0CFBB2
:101140000BF7D21B03FB0CF761EB07010CFB0EF74F
:10115000B0EB074072EB17420CFB08F734BFA2EB71
:101160000742B2EB074261EB174115EB1C154FEA42
:10117000813141EA92414FEA823242EA90424FEA9B
:1011800080304FEA0C7644F1000448EA03434EEA0B
:101190000B484FF0000EB2EB080C71EB030724BFB5
:1011A000624639464EEB0E0E4FF0000B00185241CE
:1011B00049414BEB0B0BB2EB080C71EB03077BF1D6
:1011C000000B24BF624639464EEB0E0E4FF0000B6B
:1011D0000018524149414BEB0B0BB2EB080C71EB81
:1011E00003077BF1000B24BF624639464EEB0E0E1F
:1011F00051EA020718BF46F0010616EB0E7655F1CC
:10120000000254F1000103D5BDE88901BDE8008862
:10121000BDE88901BDE80048B619524141EB010122
:10122000A3F10103704780807F7E7D7C7B7A797893
:10123000777676757473727171706F6E6E6D6C6C9B
:101240006B6A6A696868676666656464636362613D
:101250006160605F5F5E5E5D5D5C5C5B5B5A5A59BE
:10126000595858575756565555555454535352522A
:101270005251515050504F4F4F4E4E4D4D4D4C4C82
:101280004C4B4B4B4A4A4A494949484848474747CB
:101290004746464645454544444444434343434208
:1012A000424242414141002B9C4630D477002BD032
:1012B0001CB54FEA370703B44FF010004FF0100190
:1012C000BAF1000F06D0BCF1000FDCBF40F00800FF
:1012D00040F008014FF000000FBCBDE810400BF1DA
:1012E000010BBBF1010F08BF5FEA170722BF12F124
:1012F000010211F101014FF0004143F1000300F040
:10130000004043EA00007047F9D35708D0E746EAA7
:10131000064613F1400F4FEA16461FDD13F1200F6A
:10132000DFBF16430A46002120335B42BED0C3F123
:10133000200746EA064602FA07F74FEA164646EA4B
:101340000706C3F1200722FA03F201FA07F721FA90
:1013500003F14FF0000342EA0702A7E746EA02065C
:1013600046EA06464FEA164646EA0106BCBF46EA8A
:101370000646360C4FF000034FF000024FF000011C
:1013800094E72DE9804C9A46934670B491E8380072
:1013900007C831EA400C48BF34EA430C03D5FFF7D5
:1013A000E6FDFFF780FFF0BCBDE8008C2DE9804C26
:1013B0009A46934670B491E8380007C810F0804F01
:1013C00008BF13F0804F03D100F005F8FFF76BFF63
:1013D000F0BCBDE8008C20F07F4780EA030023F0DA
:1013E0007F4C07EB0C03A3F57C5300F00040A3F106
:1013F000FE0392F0000F00F0B38095F0000F00F0B4
:1014000077802DE901494FEA11404FEA144621EA5D
:10141000004800FB06FC24EA064708FB06F607FB2B
:1014200008F800FB07F718EB06484CEB164C4FEAA0
:10143000124B18EB07484FEA15464CEB174022EACF
:101440000B4E0BFB06FC25EA06470EFB06F607FBD8
:101450000EFE0BFB07F71EEB064E4CEB164C4FF047
:1014600000061EEB074E4CEB174B18EB0B0840F138
:10147000000018EB0E0B58EB000840F100008F1A2B
:101480004FF000013CBFC943661B14BFB5EB040C11
:1014900000213CBFC943F61B4FEA17444EEA8E0EAB
:1014A00027EA04454FEA1C4704FB07622CEA074C75
:1014B00005FB07F70CFB05F604FB0CFC16EB0746D7
:1014C00042EB174216EB0C4642EB1C421BEB0606A6
:1014D00058EB0202414146EA9E0601D5BDE801896A
:1014E000B619524141EB0101A3F10103BDE80189A5
:1014F0004FEA14454FEA114724EA054621EA074C12
:1015000005FB07F406FB07F70CFB06F105FB0CFCDB
:1015100011EB074144EB17444FEA124711EB0C4122
:1015200044EB1C4422EA074C05FB07F206FB07F7D5
:101530000CFB06F605FB0CFC16EB074642EB1742CC
:1015400016EB0C4642EB1C456A1854F1000148BFEB
:101550007047B619524141EB0101A3F101037047F5
:1015600095F0000F37D04FEA11424FEA144721EAB5
:10157000024624EA074C02FB07F106FB07F70CFBC7
:1015800006F402FB0CFC14EB074441EB17414FEA55
:10159000154714EB0C4441EB1C4125EA074C02FBB8
:1015A00007F506FB07F70CFB06F602FB0CFC16EB37
:1015B000074645EB174516EB0C4645EB1C42121946
:1015C00051F1000148BF7047B619524141EB01018A
:1015D000A3F1010370474FEA14454FEA114724EA8B
:1015E000054621EA074C05FB07F106FB07F70CFB54
:1015F00006F24FF0000605FB0CFC12EB074241EB34
:10160000174112EB0C4251EB1C4148BF7047921836
:1016100041EB0101A3F101037047FEE770470000B1
:10162000064A074902284FF0010004D09062886FF3
:10163000486701F005B99061C86FF9E700040048F8
:101640008000002030B50022214C13464FF4FA559B
:10165000181990F8AC071044401CC2B2284603F099
:1016600051FA5B1CDBB25F2BF2D394F8AC0700217C
:10167000174B0C3393F8AC37034415480E3090F8F1
:10168000AC0703441248463090F8AC0703441048B6
:10169000473090F8AC0703440D48503090F8AC0741
:1016A00003440B48513090F8AC071844C01CC0B23A
:1016B00002B9212210B1FF2808D000E00121002347
:1016C000194300D04D2242EA002030BD0123F7E744
:1016D00000F0FF1FFEE7000070B5124C802525606A
:1016E000962003F00FFA40222260962003F00AFAB7
:1016F0000C4B0C4E1033083E07E01A60962003F0A6
:1017000001FA2260962003F0FDF930680006F4D556
:101710001D60962003F0F6F91A60BDE8704096202F
:1017200003F0F0B918040048094800B580220260AF
:10173000962003F0E7F9064B4020103B18609620F6
:1017400003F0E0F91A6096205DF804EB03F0DAB9D3
:1017500028040048F0B5154C00238027134E1034A0
:1017600005464022280601D5376000E02760962014
:1017700003F0C8F93260962003F0C4F922606806CD
:101780005B1C050EDBB2082BECD3962003F0BAF9F4
:101790003260962003F0B6F90448083800682260E9
:1017A00040F3C0102760401CF0BD00001804004842
:1017B00030B5054600240AE004F15A00C1B2042005
:1017C00003F07CFDFF2006F0C1FE641CE4B2AC42D5
:1017D000F2D930BD10B5002404F15A00C1B2042082
:1017E00003F06CFD002006F0B1FE641CE4B2272C6F
:1017F000F2D310BD70B50024184A0621184800F035
:10180000EFF84FF0A042D2F8080140F00100C2F812
:10181000080100234FF4AF75D2F8080140F004002E
:10182000C2F808010F2003F06DF9D2F84001A04280
:1018300000DD04465B1CAB42EEDBB4F10C0000D5CE
:10184000002007F0D6FA9FED071B53EC112B07F091
:10185000DFF8BDE8704007F06FBA00001000C0105C
:1018600000010050CDCCCCCCCCCCF83F0D49CA689F
:10187000D207FCD1CA6893064FF0200200D5CA6097
:101880000B6943F002030B614861086940F04000B6
:101890000861C8688006FCD5CA60086920F00200AB
:1018A0000861704700200240F0B5114CE368DB0787
:1018B000FCD1E3684FF020059B0600D5E560236965
:1018C00043F00103236100230AE0C718C65C7F7858
:1018D00006EB0726CE52E668B606FCD5E5609B1CF3
:1018E0009342F2D3206920F001002061F0BD000096
:1018F0000020024030B54FF0A0444B68A46800229D
:101900000E4D04F00104AD6805F001052C4302D032
:101910000122104630BD0A4D53B10C681C43D1E979
:1019200002310B4381681C4329400C438460F0E77B
:10193000836809682B400B438360EAE7000100508D
:10194000E030FCFF816821F0405181608168034AEA
:10195000114041F08051816070470000C0FFFF7F5F
:1019600030B58368002213F0010F02D00122104627
:1019700030BDD1E9003423438968C46844F2380596
:10198000AC4321430B43C360F1E7000070B54C68E2
:101990008368002213F0010F02D00122104670BDAF
:1019A000002C0E4B0C6807D08D682C43D1E90356F0
:1019B00035432C434D6904E0CD682C43D1E90456EE
:1019C00035432C43C5681D402C43C4604968036BF4
:1019D00023F00F030B430363E0E700003CC0F0FF7C
:1019E00010B54FF4407494FAA4F401F44073B4FABF
:1019F00084F4E34000EB8300036B01F01F011F241C
:101A00008C40C2F38462A3438A401343036310BD36
:101A100070B54FF0007494FAA4F401F00073B4FAB6
:101A200084F4E34000EB830043694FF0F87494FAC8
:101A3000A4F501F0F871B5FA85F521FA05F5072648
:101A4000AE4094FAA4F4B4FA84F4E140B3438A407B
:101A50001343436170BD000030B550F8B04F064BE2
:101A600002F0180201EA0305D3400B40AC4323F017
:101A700001010C43046030BDFEFF0700044908B5B6
:101A80004A6902434A6149690140009108BD00006A
:101A900000100240044908B5CA690243CA61C96915
:101AA0000140009108BD00000010024070B5002404
:101AB00001F010010123556806688B40B3430ED036
:101AC0007DB113682B43D2E9025215432B430268C0
:101AD0008B4040F6FA758D40AA4313430AE0012477
:101AE00009E00368FA258D40AB431568D2681543B9
:101AF0008D402B430360204670BDF0B50A680F2669
:101B000092FAA2F2B2FA82F303248EE001259D40FC
:101B10002A407ED04D68012D01D0022D20D18D6844
:101B2000876892FAA2FCBCFA8CFC4FEA4C0C04FACF
:101B30000CFC27EA0C0792FAA2FCBCFA8CFC4FEAD8
:101B40004C0C05FA0CF52F438760CF680D68D0F870
:101B500004C02CEA050C7D434CEA050CC0F804C017
:101B60000F69D0F80CC092FAA2F5B5FA85F54FEAE4
:101B7000450E04FA0EF52CEA050C92FAA2F5B5FA18
:101B800085F56D00AF404CEA070CC0F80CC04D68FD
:101B9000022D33D192FAA2F5B5FA85F5082D15D2AA
:101BA000D1F814C0056A92FAA2F7B7FA87F7BF0016
:101BB00006FA07F7BD4392FAA2F7B7FA87F7BF0014
:101BC0000CFA07FC45EA0C05056217E0D1F814E0B1
:101BD000476A150A95FAA5FCBCFA8CFC4FEA8C0CF6
:101BE00006FA0CFC95FAA5F5B5FA85F5AD0027EADD
:101BF0000C070EFA05FE47EA0E0747624D680768B4
:101C000092FAA2FCBCFA8CFC4FEA4C0C04FA0CFED3
:101C100000E009E092FAA2F2B2FA82F2520027EA58
:101C20000E0795402F4307605B1C0A6832FA03F5E4
:101C30007FF46CAF0020F0BD0069814301D000202B
:101C40007047012070474FF47A71B0FBF1F14FF00B
:101C5000E020491E41610021816105210161704739
:101C600001490860704700002C0200200A7B8B6845
:101C70001A434B6822F480621A430B6822F4006214
:101C80001A43CB8922F480521A430B6922F4005282
:101C90001A434B6A22F480421A4322F400421A4348
:101CA0004B6922F470221A43084B98420BD10B6AFD
:101CB00022F470021A438B6922F080721A43C969B8
:101CC00022F000720A43426400207047002C014059
:101CD000F0B502681A4B1B4F4FF0804C984203D06E
:101CE000604501D0B84203D14C6822F07002224313
:101CF000154C164D164E984209D0604507D0B84293
:101D000005D0A04203D0A84201D0B04203D1CF6891
:101D100022F440723A4302608A68C2620A88826290
:101D2000984205D0A04203D0A84201D0B04201D1D0
:101D300009690163416941F0010141610020F0BD81
:101D4000002C0140000400400040014000440140DC
:101D5000004801402DE9F047DFF8D8C20023B64C17
:101D6000B64DB74EB74F4FF001084FEA3C69B1F599
:101D7000805F7DD007DC01290CD0102948D0B1F557
:101D8000807F76D18CE0B1F5803F73D0B1F5801FB4
:101D90006FD121E1016A21F001010162D0F820A098
:101DA0004168D0F81880A04228F0030808EA0C081F
:101DB000D2F800C048EA0C09D2F810802AF0020CD0
:101DC0004CEA080CD2F804802CF0010C4CEA080C08
:101DD00005D0A84203D0B04201D0B84212D1556913
:101DE0002CF0080444EA8504956824F0040444EACD
:101DF000850C946921F480712143D46921F4007128
:101E000041EA44014160C0F81890D16841630EE195
:101E1000016A21F010010162D0F820A0D0F804C0BE
:101E20008169D2F8008021F4407101EA090141EA98
:101E30000829D2F810802AF0200141EA0811D2F8CE
:101E4000048021F0100141EA0811A04205D0A84207
:101E500003D0B04201D0B84217D1546921F08001BB
:101E600041EA8411946821F0400141EA841102E0C2
:101E700055E012E083E095692CF4806444EA85041F
:101E8000D56924F4006444EAC50CC0F804C0C0F865
:101E90001890D2688263016298464046BDE8F08798
:101EA000016A21F480710162D0F820904168D0F875
:101EB0001C80A04228F0030808EA0C08D2F800C0F1
:101EC00048EA0C0AD2F8108029F4007C4CEA082C6D
:101ED000D2F804802CF4807C4CEA082C05D0A8426F
:101EE00003D0B04201D0B84213D155692CF400643C
:101EF00044EA8524956824F4806444EA852C946936
:101F000021F4805141EA0411D46921F4005141EADD
:101F100044114160C0F81CA0D168C16387E0016A28
:101F200021F480510162D0F820A04168D0F81CC093
:101F3000D2F800802CF4407C0CEA090C4CEA082909
:101F4000D2F810802AF4005C4CEA083CD2F80480F5
:101F50002CF4805C4CEA083CA04205D0A84203D097
:101F6000B04201D0B84204D1946921F4804141EAE1
:101F700084114160C0F81C90D168016457E0016A87
:101F800021F480310162D0F82080416DA04201EA45
:101F90000C01D2F800C041EA0C0128F4003CB2F870
:101FA00010804CEA084CB2F804802CF4803C4CEAD7
:101FB000084C05D0A84203D0B04201D0B84206D1A7
:101FC0004468956924F4803444EA052444604165FA
:101FD000D168826D81652AE0016A21F48011016275
:101FE000D0F820C0416DD2F8008001EA090141EA31
:101FF0000821B2F810802CF4001C4CEA085CB2F8FE
:1020000004802CF4801C4CEA085CA04205D0A84255
:1020100003D0B04201D0B84206D14468956924F497
:10202000802444EA852444604165D168C165C0F8D4
:1020300020C031E78FFFFEFF002C0140004001402F
:10204000004401400048014008B54FF0E0210A6912
:102050000092421C00D0401C0A69D20300D5401EE9
:102060000028F9D108BD000030B593B000241094C9
:102070001194182168461294FEF7BCFA0C940D9442
:102080000E94182106A80F94FEF7B4FA4FF0805072
:10209000FFF7F4FC4FF40030FFF7F0FC022006904D
:1020A0000320079006A90A944FF09040FFF725FD02
:1020B0004FF0A0451094119410A928461294FFF7F0
:1020C0004FFC0094019401200294CDE903400003E9
:1020D000059069462846FFF759FC0C940CA9144852
:1020E0000D94FFF707FC2846FFF72CFC1148124916
:1020F0000068B0FBF1F000EB800040000A21B0FB6B
:10210000F1F100E0491E0029FCD10C4C06212246C9
:102110002846FFF765FC002221462846FFF778FC99
:102120007F2221462846FFF797FC13B030BD000000
:10213000000300502C020020400D03000400600842
:1021400030B58FB000240C940D94182106A80E947D
:10215000FEF750FA18216846FEF74CFA4FF080500F
:10216000FFF78CFC4FF40030FFF788FC4FF4802021
:10217000FFF784FC80200325CDE90005694604941F
:102180004FF09040FFF7B9FC0420CDE90005694607
:1021900004941D48FFF7B1FC1C4D0C940D940CA940
:1021A00028460E94FFF7DCFB069407940120089460
:1021B000CDE9094000030B9006A92846FFF7E6FB8E
:1021C0002846FFF7BFFB124812490068B0FBF1F048
:1021D00000EB800040000A21B0FBF1F100E0491E55
:1021E0000029FCD10C4C062122462846FFF7F8FBBB
:1021F000002221462846FFF70BFC7F222146284675
:10220000FFF72AFC0FB030BD000400480001005069
:102210002C020020400D03001000C01010B58AB041
:102220000024009401940294182104A80394FEF75A
:10223000E1F94FF00050FFF72DFC4FF40030FFF7AD
:102240001DFC302004900320059004A908944FF051
:102250009040FFF752FC00F06BFF0022114600F0A7
:10226000E3F90146362000F06BFF362000F052FF04
:102270003820CDE9000403940C4C6A460A492046F4
:10228000FFF714FC206820F0040020600220039077
:102290006A4607492046FFF709FC206820F48020A1
:1022A00020600AB010BD0000010010020074004060
:1022B0001200431510B58AB00024069407940894C0
:1022C000182168460994FEF795F94FF08060FFF7F2
:1022D000E1FB4FF40030FFF7D1FB402000900320DA
:1022E0000190694604944FF09040FFF706FC3820B7
:1022F000CDE906040220074C099006AA04492046AD
:10230000FFF7D4FB206820F0040020600AB010BD65
:1023100001001002009800402DE9F04387B0182119
:102320006846FEF767F94FF40020FFF7A7FB4FF46C
:102330008000FFF7A3FB4FF40030FFF79FFB4FF443
:102340008020FFF79BFB24484FF400518162DFF8A7
:102350008C904CF2F906C9F828604FF0904848F28A
:102360000817C8F82870009101250024CDE9015410
:10237000039469460494FFF7C0FB0420CDE90004F0
:10238000694604954046FFF7B8FB0096CDE9015435
:102390000394694648460494FFF7AFFB4FF470502E
:1023A000CDE90004694604954846FFF7A6FB00976F
:1023B000CDE901540394694640460494FFF79DFB20
:1023C0006802CDE90004694648460494FFF795FB8E
:1023D00007B0BDE8F0830000000800480004004892
:1023E000F0B59FB0142118A8FEF704F920210AA81F
:1023F000FEF700F928216846FEF7FCF8182112A81C
:10240000FEF7F8F82F48816941F400318161806955
:10241000002400F400301D9040F22B10ADF8600055
:10242000401CCDE91940284E1B9418A930461C9435
:10243000FFF74EFC306840F08000306023480178A0
:10244000214818300D182868204F082109373A789C
:102450009140084328606020CDE90A040C940D9453
:102460000E940F9410940AAA012130461194FFF79C
:1024700071FC28683A7804219140884328600094D0
:102480007014CDE9040440008DF80C4009900194CB
:102490000294ADF80E4069463046FFF7E7FB4FF473
:1024A0008020FFF7EBFAB01512900220CDE913045B
:1024B0000120CDE9164012A915940548FFF71DFB30
:1024C0001FB0F0BD0010024000440140C29400085B
:1024D0000004004810B586B014216846FEF78AF85B
:1024E0000120FFF7D7FA00F023FE0222114600F088
:1024F0009BF801461C2000F023FE1C2000F00AFE81
:1025000045F6BF50ADF8000000202721CDE90101BC
:102510004FF08044039069462046FFF7D9FB2068BE
:1025200040F080002060A06806490840A060606814
:1025300020F070006060A06820F08000A06006B00D
:1025400010BD0000F8BFFEFF10B586B0142168462C
:10255000FEF750F80220FFF79DFA00F0E9FD002297
:10256000114600F061F801461D2000F0E9FD1D2034
:1025700000F0D0FD0020ADF80000E021CDE9010120
:102580000B4C039069462046FFF7A2FB206820F021
:1025900080002060A06807490840A060606820F0C3
:1025A00070006060A06820F08000A06006B010BDE0
:1025B00000040040F8BFFEFF10B586B01421684645
:1025C000FEF718F81020FFF765FA00F0B1FD0122C0
:1025D000114600F029F80146362000F0B1FD362002
:1025E00000F098FD0920ADF800000020019040F2B5
:1025F000DC500B4C029069462046FFF769FB2068CF
:1026000020F080002060606820F0700040F0200022
:102610006060A06820F08000A06006B010BD0000DF
:1026200000100040FEE7FEE730B500F00703C3F1FD
:102630000704042C00D90424181D072801D2002304
:1026400000E0DB1E012505FA04F0401E084098401A
:102650009D406D1E1540284330BD000070B500221E
:1026600001264849032305240725052805D24E7075
:102670008B70CC700D714A7105E00ED14A708E706E
:10268000CB700C714D718A71CA710A724A728A726A
:10269000CA720A734A738A7370BD06281ED007284F
:1026A00023D0082829D0092830D00A2838D00B2870
:1026B00041D00C284BD00D2856D00E28ECD14A70B2
:1026C0008A70CA700A714A718A71CA710A724A7232
:1026D0008A72CE720B734C738D7370BD4A708A70A0
:1026E000CE700B714C718D71CEE74A708A70CA70D2
:1026F0000E714B718C71CD71C7E74A708A70CA70C8
:102700000A714E718B71CC710D72BFE74A708A707D
:10271000CA700A714A718E71CB710C724D72B6E734
:102720004A708A70CA700A714A718A71CE710B72CE
:102730004C728D72ACE74A708A70CA700A714A7125
:102740008A71CA710E724B728C72CD72A1E74A7097
:102750008A70CA700A714A718A71CA710A724E729D
:102760008B72CC720D7395E74A708A70CA700A71C9
:102770004A718A71CA710A724A728E72CB720C7374
:102780004D7388E75302002030B5092800D909208D
:10279000062101EB4004C0F10A05E1B2F62015FB69
:1027A00000F040B205F068FD05EBC500E1B2BDE800
:1027B000304040B205F060BD15481649C26E0A604F
:1027C000154B511CB3FBF1F1490940F6340391FB61
:1027D000F3F380F83B3000F58073596190F82730AF
:1027E0004FEA4111022B01D26C2300E0362391FB0A
:1027F000F3F121F01F0146238167B1FBF3F1C167BB
:102800000720B2FBF0F002498031086070470000F9
:10281000000000202C04004000D8B80570470000DC
:102820000449497A494200EBC1200349084490F821
:10283000000C70470000002000F000087047000006
:1028400010B5044C606F05F0B9FD606FBDE8104035
:1028500005F080BD8000002010B5094C606F05F0C8
:10286000ADFD606F05F076FDA4F18000462190F883
:102870003A0010FB01F0BDE8104005F015BE000065
:102880008000002070B5403046B20820A0EBD10592
:1028900001F007008024C440F1B2E8B202F00EFD5E
:1028A000054806EB46010144485D2043C0B2485547
:1028B000BDE8704005F04ABEB809002070B5082494
:1028C0000E463E2801DD012100E0002110F13E0FFF
:1028D00001DA012200E00022114336D1403045B236
:1028E000E9B2082002F0EAFC002005F02FFEE9B270
:1028F000072002F0E3FC002005F028FEE9B20620E4
:1029000002F0DCFC002005F021FE072E07D9E9B219
:10291000082002F0D3FCFF2005F018FE07240F2E3C
:1029200007D9E9B2072002F0C9FCFF2005F00EFE2E
:102930000624E9B2204602F0C1FC044906F0070073
:10294000085CBDE8704005F001BE70BD300200209B
:102950007047000070B52D48016821F0070141F073
:1029600002010160016801F007010229FAD1284C37
:10297000206840F4803020602068C0F34040002888
:10298000FAD0606A40F001006062606AC0F3400003
:102990000028FAD061684FF4803021F4741141F4BA
:1029A00024116160E16A60F30301E162206840F094
:1029B000807020602068C0F340600028FAD0606812
:1029C00020F0F0006060606820F4E06040F4806017
:1029D0006060606820F460506060606820F0030010
:1029E00040F002006060606800F00C000828FAD136
:1029F000084D2846FFF727F92846FFF731F9E06A26
:102A000020F4F87040F49870E06270BD002002403D
:102A10000010024000D8B8050248016841F4700176
:102A20000160704788ED00E02DE9F05F4FF08041D4
:102A30006FF001000861B64D287A08B1401E287277
:102A400095F821004FF0010A00287CD1B14E0024F6
:102A5000274606F1840800BF56F8240095F82B108D
:102A600000EE100A2046B8EEC00A02F005FCBDEEEA
:102A7000C00A10EE101A48F8241046F82470641C9E
:102A8000E4B2202CE8D3FF2185F821109FEDA20AA3
:102A9000A24EDFF88CC2A6F1800486ED060AE7613B
:102AA00000233A463946C1460CF1840BC4F818702D
:102AB00059F823000CEB830800EE100AF8EEC00A68
:102AC00000EE100AB8EEC01A96ED060A00EE810A72
:102AD00086ED060A00EE100A98ED001AF8EEC00A1C
:102AE00000EE102AB8EEC00A00EE810ABDEEC00A60
:102AF00010EE102A00EE100A0BEB83005B1CF8EEC0
:102B0000C00A00EE101A90ED001ADBB2B8EEC00A4F
:102B1000202B00EE810ABDEEC00A10EE101AC7D3BA
:102B2000C4E9062196ED060ADFED7E0A20EE200AB2
:102B300010EE100A06F048FC41EC100B01F028F8EA
:102B400051EC100B00E0DDE005F07CFE00EE100A19
:102B500086ED060AD5ED1F0AF8EE600A80EE201A0F
:102B6000BCEEC10A85ED1C0AA0692063E1696163BE
:102B7000EA79012A03D095F82720022A04D2C4F862
:102B800020A0C4F824A010E0E26B121A00D5524233
:102B9000032392FBF3F2521C6262A26B521A00D51D
:102BA000524292FBF3F2521C2262E26B636A904241
:102BB00001DD1A4400E0D21AE263A26B236A91425B
:102BC00001DD1A4400E0D21AA26395F820201AB160
:102BD00085F82070C4E90E10E26B801A2063A26BA6
:102BE000891A616395F8271001290CD000EE100AAC
:102BF000B8EEC00A02F006FABDEEC00A84ED140A6F
:102C000094ED0D0A72E095F83810012904D00229DC
:102C100013D0032922D035E000EE100AB8EEC00A26
:102C200002F08AF8BDEEC00A84ED140A94ED0D0A94
:102C3000B8EEC00A02F0FEF820E000EE100AB8EE8E
:102C4000C00A02F0A3F8BDEEC00A84ED140A94EDA8
:102C50000D0AB8EEC00A02F017F90FE000EE100AF4
:102C6000B8EEC00A02F0BCF8BDEEC00A84ED140A4A
:102C700094ED0D0AB8EEC00A02F030F9BDEEC00ABC
:102C800084ED150A95F82C0018B10021042815D000
:102C900000E001210022114312D094ED140AB8EE95
:102CA000C00A02F067F9BDEEC00A84ED140A94ED83
:102CB000150AB8EEC00A02F0EDF91BE00122EAE7BE
:102CC000012803D00021032820D000E001210020AA
:102CD000014313D094ED140AB8EEC00A02F092F941
:102CE000BDEEC00A84ED140A94ED150AB8EEC00AD0
:102CF00002F018FABDEEC00A84ED150A206DA0623C
:102D0000606DE06285F835A0BDE8F09F0120DFE747
:102D1000000000206C0300200000000000010020E3
:102D2000640200200000003D30B516480022026019
:102D30001548164B164C8178491C01F01F01817013
:102D400053F821302360114B124C843B53F821304F
:102D5000236090F82130002B13D00F4B4FF0A0458B
:102D600053F821402D6C2C44A4F2FD7443F821400B
:102D7000416F491C4167836F994202D380F821203B
:102D8000426730BD1004004000000020F80400201D
:102D900014740040089800406C0300200B496FF049
:102DA000010008610A48017A002909D110F8421F80
:102DB000CA0701F101010170064802D0002101603B
:102DC0007047034980314969F9E70000001000406D
:102DD000000000200874004070B51820FFF720FDA7
:102DE000374C84F8310005202B34FFF719FDA07013
:102DF0000620FFF715FD04F82B091420FFF710FD3E
:102E00002F4D8035A8671320FFF70AFD18B1A86F72
:102E100000F58070A8671A20FFF702FDE867192007
:102E2000FFF7FEFC18B1E86F00F58070E867FFF768
:102E300007FD94F82C20234848F201011023C2B169
:102E4000012A16D0022A17D00126032A18D00A21F7
:102E5000042A18D0052A19D0062A21D0072A0AD117
:102E600048F20301816023766C6F0A2C1DDB0A3C5B
:102E70001DE08160237670BD81600820207670BDE2
:102E80008160267670BD48F25F020BE048F20F02C7
:102E900082602176032084F8380084F82D6070BDAC
:102EA00049F6DF028260217670BD04F5AF742046DA
:102EB00005F084FA2046BDE8704005F04BBA0000EA
:102EC000000000200001002010B5104A0621104823
:102ED000FEF786FD4FF0A042D2F8080140F0010055
:102EE000C2F80801142002F5847201F00BFE10688C
:102EF00040F0040010601A2001F004FE906B0549B8
:102F000091F8331090FBF1F010BD0000001060321A
:102F10000001005000000020FEE7000070B50446EC
:102F200001F0BCFD1EA12148FDF7D4F91F4A142170
:102F3000032001F0ABFE4FF47A7001F049FD012C43
:102F400001D105F0E5FB1B48194941601A49416070
:102F50001A4800F057F8194C194D093C607A404264
:102F600005EBC020FEF782FC607A1022404205EBA0
:102F7000C02104F22910FEF797FC607A1049404204
:102F8000103101EBC021102204F23910FEF78CFC45
:102F90004FF4FA70FFF758F8BDE8704001F07EBDBD
:102FA0002020575249544520212020003C02002077
:102FB0002301674500200240AB89EFCD09000020C6
:102FC00000FC00080B4910B5094A4A600A4A4A60E9
:102FD000012801D105F0FCFB084C2046FEF746FC19
:102FE0002146BDE8104008220548FEF75DBC000000
:102FF0002301674500200240AB89EFCD00D40008D3
:103000002101002010B5054C2046FEF72FFC21467B
:10301000BDE8104002220248FEF746BC00DC000872
:103020000900002070B50E460546FEF755FB4FF42B
:103030007A74204601F066FD5820FEF78BFB20468F
:1030400001F060FD2846FEF785FB204601F05AFDA1
:103050003046FEF77FFBBDE87040FEF765BB000021
:103060001E4800B590F80014FF292ED05FF0000133
:1030700090F8000458B3002001432ED01748801C5C
:1030800090F80014FF2924D05FF0000190F80004AC
:1030900008B30020014320D0FEF7D4FA104966227D
:1030A000A1F221134A7000228A709A74030ACB702D
:1030B00048710A71A1F1A1008A71C2605720C871DC
:1030C00010465DF804EBFFF77DBF0121D0E701203A
:1030D000D2E70121DAE70120DCE700BD03D00008D8
:1030E0002101002003B401984100009850EAC1205A
:1030F00018BF04204A0D18BF40F0010040F2FF72D3
:10310000B2EB515F08BF40F00200012808BF052064
:1031100002B07047002809DB00F01F020121914036
:103120004009800000F1E020C0F800117047000065
:1031300002480068C0F30220704700000CED00E078
:103140000907090E002804DB00F1E02080F80014D4
:10315000704700F00F0000F1E02080F8141D704768
:1031600070B59B482DED020B2DED068B079D25F0CC
:103170000044A04218DC9748844202DC0AD1069839
:1031800040B19DED060BBDEC068B02B0BDE8704072
:1031900001F026BB002DCCBF9FED8F0B9FED900B58
:1031A000BDEC068B02B070BD8F48A04215DD8F4884
:1031B000A042D8BF4FF0FF3458DD9DED060B51EC17
:1031C000100BFFF78FFF042808BF01F02DFB9DEDCA
:1031D000060BBDEC068B02B070BD9DED060B51ECED
:1031E000100B01F09DFDCDE9060181489FED828B1A
:1031F000A0423CDD8248A0421FDD00249FED82AB4F
:103200009DED060B53EC1A2B51EC100B05F04CFB0B
:103210009DED060B41EC190B53EC1A2B51EC100BE6
:1032200005F012FE53EC182B05F0E4FF53EC192BBC
:1032300005F0EEFBCDE9060149E09DED060B01240A
:1032400053EC182B51EC100B05F02EFB9DED060BEB
:1032500041EC190B53EC182B51EC100B05F0CAFF85
:1032600053EC192B05F0D4FBCDE906012FE068489B
:10327000A0421FDD02249FED689B9DED060B53ECE1
:10328000192B51EC100B05F0DFFD53EC182B05F05A
:103290000BFB9DED060B41EC180B53EC192B51EC7D
:1032A000100B05F0A7FF53EC182B05F0B1FBCDE98F
:1032B00006010CE09DED060B032453EC102B9FED53
:1032C000580B51EC100B05F0A3FBCDE906019DED69
:1032D000060B53EC102B51EC100B05F0B5FD41EC37
:1032E000180B53EC182B05F0AFFD41EC190B4E48B1
:1032F0000621B0EE490AF0EE690A784400F09CFF1E
:1033000053EC182B51EC100B05F09EFD41EC180B03
:103310004648B0EE490AF0EE690A0521784400F00B
:103320008BFF53EC192B51EC100B05F08DFD41EC8C
:10333000100B51EC180B53EC102B002C0EDA05F08F
:10334000B3FA9DED061B53EC112B05F07DFD9DEDB1
:10335000061B53EC112B05F075FE35E005F0A4FAC1
:103360009DED061B53EC112B05F06EFD41EC100B8F
:103370002F48784400EBC40090ED001B51EC100B7B
:1033800053EC112B05F036FF9DED061B53EC112B72
:1033900005F030FF41EC100B2648784400EBC400E8
:1033A00090ED001B51EC100B53EC112B05F04AFE75
:1033B00041EC100B002DA2BFBDEC068B02B070BD1E
:1033C00051EC100B05F032FA41EC100B01E7000054
:1033D000000010440000F07F182D4454FB21F93FF9
:1033E000182D4454FB21F9BF0000DC3F0000203EB3
:1033F0000000F33F00000000000000000000F03F6C
:103400000000E63F00000000000000000000004057
:103410000080034000000000000000000000F83FB2
:10342000000000000000F0BF727700002877000065
:10343000B27600006A76000070B56F4E2DED040B79
:103440002DED048B82B0DDF824C0DDE907235C425A
:103450002CF000411C4341EAD474069D22F0004048
:10346000B44205D86C422C4340EAD474B4420BD920
:103470009DED081B9DED060B02B0BDEC048B04B066
:10348000BDE8704001F0B6B9ACF14054A4F17F64DE
:103490001C430BD0022404EAAC7444EAD274054302
:1034A0009FED578B9FED582B07D015E09DED060B38
:1034B00051EC100B01F0CFF942E0002C11BF012CB0
:1034C0009DED060B02B0BDEC048B04BF04B070BDD3
:1034D000022C38D0032C3BD00B439FED4D1B9FEDAE
:1034E0004E0B0AD0B14218D1B04209D121F080412F
:1034F00020F08040099107900FE0002A15DA10E0D3
:10350000474B7B44002C08BF93ED000B0DD0012CE2
:1035100010D0022C17D0032C1AD0B0421DD1002A93
:1035200003DAB0EE410AF0EE610A02B0BDEC048BA2
:1035300004B070BD93ED000B51EC100B05F076F963
:1035400041EC100BF1E7B0EE480AF0EE680AECE748
:10355000B0EE420AF0EE620AE7E7401A00159FED6E
:10356000329B3C28C8BF8DED000B17DCBCF1000F6F
:10357000BCBF10F13C0F8DED009B0FDB9DED080BE8
:1035800053EC102B9DED060B51EC100B05F040FA9F
:1035900001F0C6FB01F05FF9CDE90001B4B1012CE7
:1035A00010D0022C9FED220B53EC102B9DED000B45
:1035B00051EC100B19D005F01DFE53EC182B05F043
:1035C00019FEBDE7019880F0004001909DED000BD1
:1035D00053EC192B51EC100B05F072FB04BF0220C9
:1035E000FDF737F89DED000B9FE705F003FE53EC68
:1035F000182B05F027FDA3E70000F07F0000000076
:10360000182D4454FB210940182D4454FB2109C0B6
:10361000182D4454FB21F9BF182D4454FB21F93FC8
:10362000CA7500000000000000000000000000005B
:10363000075C143326A6A13C10B52F499FED2C1B27
:103640002DED020B84B0059820F000408842D8BFD1
:103650009DED040B2DDD2949884209D1049840B91C
:103660004FF00100FCF7F5FF01F0CEF806B010BDF9
:1036700005DB9DED040B01F0B3F806B010BD684604
:103680009DED040B00F004FB10F0030004BF9DED62
:10369000021B9DED000B0CD001280ED09DED021BEE
:1036A0009DED000B022817D0012000F041FE06B06E
:1036B00010BD00F009FD06B010BD9DED021B9DED93
:1036C000000B012000F034FE51EC100B05F0AEF8B9
:1036D00006B041EC100B10BD00F0F6FC51EC100BE5
:1036E00005F0A4F806B041EC100B10BD000000007E
:1036F0000000000000000000FB21E93F0000F07F17
:1037000070B5D94B00242DED020B2DED108BDDE9AA
:103710001010984205DA20F000429A4201D809D1EF
:1037200041B19DED100BBDEC108B02B0BDE87040B7
:1037300001F056B8B0F5801F26DA11430BD00028EF
:1037400013DA0120FCF785FFBDEC108B02B0BDE859
:10375000704001F059B80220FCF77BFF01F028F817
:1037600051EC100B05F062F89EE06FF035049FED10
:10377000C00B53EC102B9DED100B51EC100B05F012
:1037800063FBCDE91001084604EB2051C0F313049C
:10379000B948A1F2FF31204400F4801080F07F622C
:1037A00082F04052224301EB20559FEDB50B119260
:1037B00053EC102B9DED100B51EC100B05F01AFD86
:1037C00041EC180BA01CC0F313009FEDAFDB9FED85
:1037D000B0EBB14E7E4403286CD296ED000B51EC59
:1037E000180B53EC102B05F06BFA1DD1002D01BF07
:1037F00096ED000BBDEC108B02B070BD284605F0B5
:10380000F8FA41EC180B53EC1D2B05F01DFB41ECB5
:10381000190B53EC1E2B51EC180B05F015FB53EC58
:10382000192B05F041F83FE09FED9D0B51EC180B73
:1038300053EC102B05F008FB9FED9B1B53EC112B59
:1038400005F000FC41EC190B53EC182B51EC180B54
:1038500005F0FAFA53EC192B05F0F6FA41EC190BC6
:10386000002D04BF53EC192B51EC180B1AD028462D
:1038700005F0BFFA41EC1A0B53EC1D2B05F0E4FAEE
:1038800053EC192B05F0DEFB53EC182B05F0B2FCC2
:1038900041EC180B53EC1E2B51EC1A0B05F0D4FA2B
:1038A00053EC182B05F0A6FCBDEC108B02B041ECDC
:1038B000100B70BD9FED7E0B51EC180B53EC102BD1
:1038C00004F0F2FF41EC100B51EC180B53EC102BF1
:1038D00005F09EF841EC190B284605F08AFA41ECF8
:1038E0001B0B53EC192B51EC190B05F0ADFA41EC05
:1038F0001A0B714853EC1A2B261851EC1A0B05F0D1
:10390000A3FA41EC1F0B6D48C4F1510404F5D72410
:10391000B0EE4F0AF0EE6F0A0321784400F08CFC01
:1039200053EC1F2B51EC100B05F08EFA41EC1C0BE5
:103930006348B0EE4F0AF0EE6F0A0421784400F0BD
:103940007BFC53EC1A2B51EC100B05F07DFA344341
:1039500053EC1C2B04F0A8FF41EC1C0B002C4CDD9D
:103960009FED510B51EC180B53EC102B05F06CFA3A
:1039700053EC182B05F068FA41EC1A0B55B353ECD5
:103980001D2B51EC1B0B05F05FFA41EC1D0B53ECAA
:103990001C2B51EC1A0B04F087FF53EC192B05F08C
:1039A00053FA53EC1D2B04F07FFF53EC1A2B05F058
:1039B00049FB53EC182B05F01DFC41EC180B53ECA4
:1039C0001E2B51EC1B0B05F03FFA53EC182B05F0A6
:1039D00011FC69E753EC1C2B51EC1A0B04F064FF4B
:1039E00053EC192B05F030FA53EC1A2B05F02AFB97
:1039F00053EC182B05F026FB56E735B353EC1D2B83
:103A000051EC1B0B05F020FA41EC1A0B53EC1C2B6C
:103A100051EC180B05F0EEFB53EC192B05F014FAE2
:103A200053EC1A2B05F0E6FB53EC182B05F0E2FBE8
:103A300041EC180B53EC1E2B51EC1B0B05F004FA58
:103A400053EC182B05F0D6FB2EE753EC1C2B51EC56
:103A5000180B05F0CFFB53EC192B05F0F5F953ECDF
:103A6000182B05F0EFFA1FE70000F07F00000000C0
:103A70000000000000005043645F090000000000E7
:103A8000000000000000F03F763C7935EF39EA3D58
:103A90000000E0FE422EE63FF87200000000000049
:103AA000555555555555D53F000000000000E03FE5
:103AB000000000000000004086EBF9FFB27000003B
:103AC000A87000000000000010B52F499FED2C1BCE
:103AD0002DED020B84B0059820F000408842DCBF39
:103AE00000209DED040B32DD2849884209D104985D
:103AF00040B94FF00100FCF7ACFD00F085FE06B0C8
:103B000010BD05DB9DED040B00F06AFE06B010BD94
:103B100068469DED040B00F0BBF810F0030011D0D7
:103B2000012818D09DED021B9DED000B02281AD034
:103B300000F0CAFA51EC100B04F078FE06B041EC2C
:103B4000100B10BD9DED021B9DED000B012000F040
:103B5000EFFB06B010BD9DED021B9DED000B00F0CC
:103B6000B3FA06B010BD012000F0E2FB51EC100BDF
:103B700004F05CFE06B041EC100B10BD000000002C
:103B80000000000000000000FB21E93F0000F07F82
:103B900000B52DED048BB0EE409AF0EE609A83B044
:103BA00051EC190B05F05AFA41EC180B18EE100AFB
:103BB00018EE901A8DED008B002818BF01200843E5
:103BC00020F00040C0F17F6000F1E040C00F14D051
:103BD00019EE101A19EE900A8DED009B002918BFFE
:103BE0000121084320F00040C0F17F6000F1E04077
:103BF000C00F04BF0120FCF72CFDB0EE480A03B053
:103C0000F0EE680ABDEC048B00BD0000000000006F
:103C100010B51D499FED1A1B2DED020B84B00598C0
:103C200020F000408842DCBF01209DED040B21DD27
:103C30001649884209D1049840B94FF00100FCF7B9
:103C400008FD00F0E1FD06B010BD05DB9DED040BA5
:103C500000F0C6FD06B010BD68469DED040B00F0F7
:103C600017F800F001000121A1EB40009DED021BBF
:103C70009DED000B00F0F4FB06B010BD000000004D
:103C80000000000000000000FB21E93F0000F07F81
:103C90002DE9F14F04462DED020B2DED088B8AB076
:103CA0009FEDE70B80ED020B139EE74826F00045E1
:103CB00085420ADC9DED120B002084ED000B0AB05A
:103CC000BDEC088B03B0BDE8F08FE0489FEDE0ABA2
:103CD0009FEDE1BBA84247DDE14F9FEDE39B9FEDE8
:103CE000E48B9DED120B53EC1A2B51EC100B002EB4
:103CF0001CDD05F07FFA41EC100BBD4208D053ECFF
:103D00001B2B51EC100B05F075FAC4E900010BE018
:103D100053EC192B51EC100B05F06CFA53EC182BEB
:103D200005F068FAC4E900010120C8E704F0BCFD11
:103D300041EC100BBD4208D053EC1B2B51EC100B87
:103D400004F0B2FDC4E900010BE053EC192B51EC77
:103D5000100B04F0A9FD53EC182B04F0A5FDC4E9E9
:103D600000014FF0FF30AAE7C348A84279DB9DED80
:103D7000120B51EC100B00F0D3FF41EC180B9FED30
:103D8000C00B53EC102B05F05FF89FEDBF1B53ECFD
:103D9000112B04F089FD04F0CFFF074605F029F848
:103DA00041EC190B53EC1A2B05F04EF853EC182B81
:103DB00005F048F941EC180B53EC1B2B51EC190B97
:103DC00005F042F8DFF8C8A241EC100B4FEA155895
:103DD0000125FA4453EC102B51EC180B05F00AFAAC
:103DE000032DC4E900013DD0C1F30A5005EB451194
:103DF000A8EB00001139814234DA0AEB051BB0EE62
:103E000048AA9BED000BF0EE68AA53EC102B51EC86
:103E1000190B05F019F841EC1B0B51EC1A0B53EC84
:103E20001B2B05F0E7F941EC180B51EC1A0B53EC86
:103E3000182B05F0DFF953EC1B2B05F0DBF99BED9C
:103E4000020B41EC1A0B53EC102B51EC190B04F044
:103E5000FBFF53EC1A2B05F0CDF941EC100B6D1C58
:103E6000B8E70EE0002EA8BF3846BFF628AF94EDA5
:103E7000000B51EC100B04F0D9FCC4E900017842AE
:103E80001DE7C6F3130040F4801EC6F30A50A0F2EB
:103E9000F530471100F01F05C5F12000DDF848B0EE
:103EA00008900020069007900520EC467949002DE7
:103EB00007EB0002794408BF51F8221009D051F8ED
:103EC000223001EB8201AB404A68089922FA01F1E5
:103ED0001943A1FB0E26A1FB0B131A449A4234BFCF
:103EE0000123002303EB06080CEB8003D3E901A6B2
:103EF0000E448E4234BF0121002192448A4411B104
:103F0000924502D903E0924501D2012100E000214F
:103F1000C3E901A641444CF82010011EA0F10100A4
:103F2000C4DC029800F10050850F0298DDE90367B8
:103F30008000DDF8148004F05CFF41EC1A0B304681
:103F400004F06EFF9FED541B53EC112B04F07CFF2B
:103F500041EC1B0B384604F063FF9FED511B53EC03
:103F6000112B04F071FF41EC180B404604F058FF90
:103F70009FED4D1B53EC112B04F066FF41EC190B28
:103F800051EC180B53EC192B04F08EFC53EC1B2B4B
:103F900004F08AFC53EC1A2B04F086FCCDE90801EE
:103FA000002008909DED080B53EC1A2B51EC100BE0
:103FB00005F020F953EC1B2B05F01CF953EC182BE2
:103FC00005F018F953EC192B05F03CF89FED381B60
:103FD00053EC112B04F038FF9FED370B41EC180B1D
:103FE00053EC102B9DED080B51EC100B04F02CFF43
:103FF00053EC182B04F058FC9FED310B41EC180BDF
:1040000053EC102B9DED080B51EC100B04F01CFF32
:1040100053EC182B04F048FC41EC100B139810F0F3
:10402000004F06D06D4251EC100B04F0FFFB41EC49
:10403000100B284684ED000B41E600000000000054
:104040000000000000000000FB21E93F7CD9024095
:1040500000004054FB21F93F3163621A61B4D03D46
:10406000FB21F93F000000000000601A61B4D03D60
:104070007370032E8A19A33BFB2139410000000015
:1040800083C8C96D305FE43F000000000000E03FDE
:10409000026D0000506C0000000000000000103EA7
:1040A000000000000000103C000000000000103A7A
:1040B000182D4454FB21F93D3326A611460B113C23
:1040C00000000054FB21F93D10B52DED040B2DED42
:1040D000088B82B0B0EE419AF0EE619A0B9820F016
:1040E00000449FED4BABB4F1795F11DA9DED0A0B03
:1040F00051EC100B04F020FE002801BFB0EE4A0A7C
:10410000F0EE6A0A02B0BDEC088B04BF04B010BD2B
:104110009DED0A0B53EC102B51EC100B04F094FEA8
:1041200041EC180B3C480621B0EE480AF0EE680A54
:10413000784400F081F853EC182B51EC100B04F08C
:1041400083FE9DED0A0B41EC1B0B53EC192B51EC3C
:10415000100B04F079FE41EC190B53EC1B2B51ECC6
:10416000180B04F071FE53EC192B05F043F89FED8A
:104170002C0B41EC190B53EC102B51EC180B04F0E9
:1041800063FE41EC100B2848844210DA53EC192BE3
:1041900051EC100B05F02EF853EC1A2B04F052FFE3
:1041A00041EC100B02B0BDEC088B04B010BD1F48F1
:1041B000A042BCBF9FED1E1B8DED001B06DBA4F5CE
:1041C00000100190002000909DED001B51EC100BA1
:1041D00053EC112B05F00EF89DED000B41EC180B84
:1041E00053EC102B51EC1A0B05F004F841EC1A0BB0
:1041F00053EC192B51EC180B04F0FCFF53EC1A2B69
:1042000004F020FF41EC100BCCE7000000000000A0
:10421000000000000000F03F6C690000000000009A
:10422000000000000000E03F3333D33F0000E93FCF
:10423000000000000000D23F70B504462DED028B57
:104240004D1E00EBC500B0EE408AF0EE608A90EDA6
:10425000000B35F0060017D053EC182B51EC100B67
:1042600004F0F2FD41EC100B6D1E04EBC50090ED67
:10427000001B51EC100B53EC112B04F015FB41EC1F
:10428000100B35F00600E7D1022D36D0042D1CD0DE
:10429000062D1CBFBDEC028B70BD53EC182B51ECEE
:1042A000100B04F0D1FD94ED0A1B53EC112B04F01C
:1042B000FBFA53EC182B04F0C7FD94ED081B53ECEC
:1042C000112B04F0F1FA41EC100B53EC182B51ECCC
:1042D000100B04F0B9FD94ED061B53EC112B04F008
:1042E000E3FA53EC182B04F0AFFD94ED040B53EC00
:1042F000102B04F0D9FA41EC100B53EC182B51ECB5
:10430000100B04F0A1FD94ED021B53EC112B04F0F3
:10431000CBFA53EC182B04F097FD94ED001B53ECF3
:10432000112B04F0C1FABDEC028B41EC100B70BDF7
:1043300031B504462DED040B2DED0A8BB0EE41BADC
:10434000F0EE61BA0B989DED0A0B20F00040B0F141
:10435000795F0DDA51EC100BFEF7C4FE042808BF9C
:1043600000F062FA9DED0A0BBDEC0A8B05B030BD82
:1043700053EC102B51EC100B04F066FD41EC180BC4
:104380009DED0A0B53EC182B51EC100B04F05CFD67
:1043900041EC190B2C48B0EE480AF0EE680A0521F2
:1043A0007844FFF749FF9FED2ACBB0EE40AAF0EE2C
:1043B00060AA9CB353EC1C2B51EC190B04F044FD88
:1043C00041EC1C0B53EC1A2B51EC190B04F03CFD87
:1043D0009FED210B41EC190B53EC102B51EC1B0BF7
:1043E00004F032FD53EC192B04F004FF53EC182BAE
:1043F00004F02AFD53EC1B2B04F0FCFE53EC1C2BA9
:1044000004F0F8FE9DED0A1B53EC112B04F01AFE8C
:10441000BDEC0A8B05B041EC100B30BDFFE753EC4F
:104420001A2B51EC180B04F00FFD53EC1C2B04F06D
:104430003BFA53EC192B04F007FD9DED0A1B53ECDE
:10444000112B04F031FAE3E7FC67000000000000E4
:10445000495555555555C5BF000000000000E03FC7
:10446000F1B506462DED040BBD482DED0C8B8AB041
:10447000B0EE418AF0EE618A179D25F000449FED71
:10448000BABB9FEDBBCB844208DA9DED160B51EC15
:10449000100B04F051FC002800F0E980B64FA74251
:1044A00031DC002D0DDA9DED160B51EC100B04F0F4
:1044B000BDF9CDE9160151EC180B04F0B7F941EC48
:1044C000180B9FEDAF0B53EC102B9DED160B51EC21
:1044D000100B04F0B7FD53EC182B9FEDAB0BCDE99F
:1044E000040151EC100B04F085FE41EC100B53EC71
:1044F000102B9DED040B51EC100B04F0D5F99FED42
:10450000A48BCDE916019DED160B53EC102B51EC4D
:10451000100B04F099FCCDE904019DED040B53EC64
:10452000102B51EC100B04F08FFC41EC190B9A4846
:104530000621B0EE490AF0EE690A7844FFF77CFEE6
:104540009648B0EE40DAF0EE60DAB0EE490AF0EEEE
:10455000690A06217844FFF76FFE9DED041B51ECBC
:10456000100B53EC112B04F06FFC9DED040B41EC90
:104570001A0B53EC102B9DED160B51EC100B04F0A5
:1045800063FC41EC190B53EC1A2B51EC1D0B04F09E
:104590008BF953EC192B04F057FC53EC182B04F057
:1045A00083F99DED041B53EC112B04F04DFC53ECEF
:1045B000182B04F079F941EC180B9FED790B51ECB5
:1045C000190B53EC102B04F03FFC53EC182B04F0A8
:1045D0006BF941EC190B9DED160B53EC192B51ECBB
:1045E000100B04F061F941EC180BA74269DC30466E
:1045F00004F0FFFB41EC1A0B51EC180B53EC1A2B97
:1046000004F052F941EC1B0B53EC182B51EC180B36
:1046100004F01AFC53EC1B2B04F0FAF953EC192BA1
:1046200004F0E8FD9DED161B53EC112B04F00AFD80
:104630009FED5D1B53EC112B04F006FC53EC1A2B81
:1046400004F000FD41EC180B022000EAA570C0F157
:10465000010004F0CEFB53EC182B04F0F5FB00BF77
:1046600041EC100B0AB0BDEC0C8B05B0F0BD711C19
:104670001698214308430CD09DED160B012E1CBF4C
:1046800053EC102B51EC1C0B10D000BF04F0C0F900
:10469000E6E79DED160B51EC100B00F041FB41ECF1
:1046A000100B51EC1B0B53EC102BEFE751EC100BE4
:1046B000FEF718FD042808BF00F0B6F89DED160BB4
:1046C000D0E7012E04BFB0EE480AF0EE680AC9D068
:1046D0008DED048B002404949DED040B53EC102B02
:1046E0009DED160B51EC100B04F0ACFC53EC192BA8
:1046F00004F0A8FC41EC190B53EC182B51EC1C0BEB
:1047000004F086F941EC180B8DED008B00949DEDC3
:10471000040B53EC102B9DED000B51EC100B04F02F
:1047200093FB53EC1B2B04F0BFF89DED000B41EC09
:104730001A0B53EC192B51EC100B04F085FB53ECC6
:104740001A2B04F0B1F853EC182B04F07DFB9DED0F
:10475000001B53EC112B04F0A7F881E700000000C8
:104760000000303E00000000000000000000F03FAC
:10477000000000000000F0BF2894E53F00000000AA
:10478000182D4454FB21E93F075C143326A6813CD5
:1047900000000000000000008A660000A066000023
:1047A000635555555555D53F0000000000000040A9
:1047B0009FED070B10B553EC102B9FED070B51EC41
:1047C000100B04F025F941EC100B10BD00000000A7
:1047D0000000000000000000000000000000F03FAA
:1047E00010B553EC102B51EC100B04F05DF841ECBC
:1047F000100B10BD10B553EC112B51EC100B04F045
:1048000053F841EC100B10BD9FED050B10B553ECA8
:10481000102B51EC100B04F0FBF841EC100B10BD09
:1048200000000000000000009FED050B10B553ECE8
:10483000102B51EC100B04F007FB41EC100B10BDDA
:10484000000000000000001030380A2801D20120CA
:1048500070470020704710B541EC100BFEF780FC4C
:1048600051EC100B10BD000070B5474C2DED028BC4
:10487000206F64287DD90120FCF7D2FE0021084674
:1048800003F0D0FD002626656665A06E206603F065
:1048900023FF4FF4FA752846FDF7D6FBDFED3B8A80
:1048A00066664FF4B476B0EE688A00BFD4E91901A9
:1048B00003F0B8FD3C20FDF7C7FB35A13648226F59
:1048C000FBF708FD344A3221062000F0A9F9206FD9
:1048D00000EE100AB8EE400AB4EEC80AF1EE10FA83
:1048E00007D200EE100A616EE165B8EE408A5028EA
:1048F00034D3606E401D6066B042D7DB4FF4FA508F
:1049000000F066F864204FF4FA66A0660146E06D98
:1049100003F088FD3C20FDF797FB1DA11E48226F88
:10492000FBF7D8FC1C4A3221062000F079F9206FF1
:1049300000EE100AB8EE400AB4EEE80AF1EE10FA02
:1049400007D200EE100AA16E2166F8EE408A5028C8
:1049500004D3A06E1430A066B042D7DBD4E91701AF
:104960000A3103F05FFD206E6065E06D206528462A
:1049700000E005E0BDEC028BBDE87040FDF764BBD4
:10498000BDEC028B70BD00000000002000E87D47F8
:104990002D253032642D00003C020020094A92F897
:1049A0003720520012FB01F1064A8032516106495C
:1049B000B1FBF0F10548C162016841F001010160FD
:1049C0007047000000000020007C920000100040B2
:1049D00010B50C490B4A0D4C91F836108900803205
:1049E00051610949B1FBF0F0E062206840F001003C
:1049F00020606420FDF728FB206820F00100206083
:104A000010BD000000000020007C9200001000405B
:104A10002DE9F041124991F82420032A1ED091F883
:104A20003610114C491CCEB20E49B1FBF0F0E062D9
:104A3000206840F001002060094F092517F1800728
:104A400006FB05F078611E20FDF7FEFA6D1E15F0DD
:104A5000FF05F5D1206820F001002060BDE8F0815D
:104A600000000020007C92000010004010B50021E2
:104A7000094A0B4601EB4104002014442354401C16
:104A8000C0B20428FAD3491CC9B28129F2D33F200D
:104A900082F8C00010BD0000B8090020F0B50B4F2F
:104AA0004FF40046BE620024641CE0B2012100F015
:104AB00005FC0025002003F049FD6D1CEDB2842D9E
:104AC000F8D3E4B2092CEFD3BE61F0BD0004004876
:104AD000F0B50B4F4FF40046BE620624012120467C
:104AE00000F0ECFB0025002003F030FD6D1CEDB262
:104AF000842DF8D3641CE4B2092CEFD3BE61F0BD61
:104B0000000400480146491EFDD10146491EFDD161
:104B10004008401EFDD17047002104E00222521CD3
:104B20006E2AFCD3491C8142F8D370472DE9F04F1F
:104B30008A461A4981464FF400409346002688620F
:104B400026E02F38C0B21649C0EB0010002401EB5C
:104B5000C00800BF09EB0400C0B2514600F0AEFB34
:104B6000002504EB440700BF05EBC70118F801005E
:104B700003F0ECFC6D1CEDB2182DF5D3641CE4B20F
:104B8000052CE7D3761C0AF11800F6B200F0FF0AF4
:104B90001BF806000028D4D1BDE8F08F00040048BF
:104BA000E49500082DE9F04F8A461B4981464FF4F1
:104BB000004093460026886228E02F38C0B217498B
:104BC000C0EB0010002401EBC00800BF09EB04009B
:104BD000C0B2514600F072FB002504EB440700BF51
:104BE00005EBC70118F80100C043C0B203F0AEFCEA
:104BF0006D1CEDB2182DF3D3641CE4B2052CE5D383
:104C0000761C0AF11800F6B200F0FF0A1BF8060045
:104C10000028D2D1BDE8F08F00040048E4950008D8
:104C20002DE9F04F8946174983464FF400409046DE
:104C3000002588621078802801D2202600E06126B5
:104C4000DFF844A018F80500002818D0801BC7B270
:104C50004946584600F032FB07EB8701002401EB80
:104C60000A07385D03F072FC641CE4B2052CF8D32B
:104C70006D1C09F10600EDB200F0FF09E2E7BDE8A6
:104C8000F08F00000004004874A600082DE9F04FE2
:104C900091468B465FEA00084FF000043AD01E4967
:104CA0004FF40040886299F80000802801D220204B
:104CB00000E06120824629E0A0F12001DE2923D80E
:104CC000A0EB0A001549C0B2002501EB001700BF98
:104CD00008EB0500C0B2594600F0F0FA5FF000069C
:104CE00006EBC500385C03F031FC761CF6B2082EEA
:104CF000F6D36D1CEDB2022DEAD3641C0BF1080053
:104D0000E4B200F0FF0B01E0641CE4B219F8040007
:104D10000028D1D1BDE8F08F00040048749C000841
:104D200082B0CDE9000121F0004001909DED000B23
:104D300002B051EC100B7047F0EE400A9FED100AE4
:104D400010490A2001EB8002401E12ED011A10F0FA
:104D5000FF0082ED001AF5D10B4AC1ED000A00BF39
:104D600002EB8003D3ED000A01EB8003401C93EDBE
:104D7000001AC0B20B2800EE810AF1D37047000080
:104D8000000000004406002038950008F0EE400ABC
:104D90009FED100A1049082001EB8002401E12ED21
:104DA000011A10F0FF0082ED001AF5D10B4AC1ED97
:104DB000000A00BF02EB8003D3ED000A01EB800381
:104DC000401C93ED001AC0B2092800EE810AF1D30D
:104DD0007047000000000000C8060020649500082D
:104DE000F0EE400A9FED100A1049062001EB800208
:104DF000401E12ED011A10F0FF0082ED001AF5D1ED
:104E00000B4AC1ED000A00BF02EB8003D3ED000A9C
:104E100001EB8003401C93ED001AC0B2072800EE9E
:104E2000810AF1D370470000000000003407002021
:104E300088950008F0EE400A9FED100A10490A20FC
:104E400001EB8002401E12ED011A10F0FF0082ED0E
:104E5000001AF5D10B4AC1ED000A00BF02EB800336
:104E6000D3ED000A01EB8003401C93ED001AC0B2A1
:104E70000B2800EE810AF1D370470000000000000B
:104E80007006002038950008F0EE400A9FED100AE9
:104E90001049082001EB8002401E12ED011A10F0AB
:104EA000FF0082ED001AF5D10B4AC1ED000A00BFE8
:104EB00002EB8003D3ED000A01EB8003401C93ED6D
:104EC000001AC0B2092800EE810AF1D37047000031
:104ED00000000000EC06002064950008F0EE400A97
:104EE0009FED100A1049062001EB8002401E12EDD2
:104EF000011A10F0FF0082ED001AF5D10B4AC1ED46
:104F0000000A00BF02EB8003D3ED000A01EB80032F
:104F1000401C93ED001AC0B2072800EE810AF1D3BD
:104F2000704700000000000050070020889500082E
:104F3000C0F30721C0B211FB0012C11D114401FBD7
:104F40000012C01C10444FF6FF72C0B202EA0121E9
:104F50000844704730B50C460146012505EBD400E6
:104F600000F0ACF904F007008540E8B2BDE830403D
:104F700003F0ECBA30B5204A0321A2F1100000BFC3
:104F800002EB810353ED010AC3ED000A00EB81033C
:104F9000491E53ED010A11F0FF01C3ED000AEFD1E4
:104FA00082ED000ADFED150A154C012120EE200AE2
:104FB00004F1100380ED000A04EB810595ED000A71
:104FC00002EB8105D5ED000A03EB810520EE200AF6
:104FD000D5ED000A00EB8105491C95ED001AC9B218
:104FE000032900EEC10AD0ED000A30EE200A80ED60
:104FF000000AE1D930BD0000200900205BC0FF3C61
:10500000A495000830B5204A0321A2F1100000BF8A
:1050100002EB810353ED010AC3ED000A00EB8103AB
:10502000491E53ED010A11F0FF01C3ED000AEFD153
:1050300082ED000ADFED150A154C012120EE200A51
:1050400004F1100380ED000A04EB810595ED000AE0
:1050500002EB8105D5ED000A03EB810520EE200A65
:10506000D5ED000A00EB8105491C95ED001AC9B287
:10507000032900EEC10AD0ED000A30EE200A80EDCF
:10508000000AE1D930BD000060090020D315003FBF
:10509000C495000830B5204A0321A2F1100000BFDA
:1050A00002EB810353ED010AC3ED000A00EB81031B
:1050B000491E53ED010A11F0FF01C3ED000AEFD1C3
:1050C00082ED000ADFED150A154C012120EE200AC1
:1050D00004F1100380ED000A04EB810595ED000A50
:1050E00002EB8105D5ED000A03EB810520EE200AD5
:1050F000D5ED000A00EB8105491C95ED001AC9B2F7
:10510000032900EEC10AD0ED000A30EE200A80ED3E
:10511000000AE1D930BD0000400900205BC0FF3C1F
:10512000A495000830B5204A0321A2F1100000BF69
:1051300002EB810353ED010AC3ED000A00EB81038A
:10514000491E53ED010A11F0FF01C3ED000AEFD132
:1051500082ED000ADFED150A154C012120EE200A30
:1051600004F1100380ED000A04EB810595ED000ABF
:1051700002EB8105D5ED000A03EB810520EE200A44
:10518000D5ED000A00EB8105491C95ED001AC9B266
:10519000032900EEC10AD0ED000A30EE200A80EDAE
:1051A000000AE1D930BD000080090020D315003F7E
:1051B000C495000870B5244E4FF40044B4624FF01B
:1051C0009045E311AB626420FFF7A6FCAB611420AD
:1051D000FFF7A2FCE22003F09DF90A20FFF79CFCF8
:1051E0002C2003F097F90A20FFF796FC2E2003F0FD
:1051F00091F90A20FFF790FC2F2003F08BF90A2089
:10520000FFF78AFC2969042088431AD05FF0250043
:1052100003F080F9812003F07DF9282003F07AF96A
:10522000A22003F077F9C82003F074F9A02003F05E
:1052300071F9402003F06EF9AF2003F06BF9B4610F
:1052400070BD2320E4E700000004004810B502F020
:10525000B3FEFDF7B1FAFDF7BFFD064C94F82D0043
:10526000FCF7DEF9FDF7F8FAD4E91401BDE81040C7
:1052700003F0D8B800000020C1F10B0100EE901A35
:105280009FED0C1A0C49F8EEE00A01EB8000D0ED1E
:10529000001A20EE811AF7EE000A70EEC10A60EEE5
:1052A000A10A41EE000AC0ED000ABDEEE00AB8EE28
:1052B000C00A70470000003D880700200A4B10B567
:1052C0004FF400429A62491EAF30CCB2C0B203F034
:1052D00021F9102000EB141003F01CF904F00F006A
:1052E000BDE8104003F016B9000400482DED088B0E
:1052F00084B0FDF72FFBFDF70FF8FCF7B5FEFCF7C8
:105300001FFFFCF71DFFFCF789FFFCF7D3FFFF48E9
:105310004CF6CC41016045F25551016006214160D7
:1053200040F6FF7181600026C1684907FCD1F7484B
:105330004AF6AA210160FDF7CDF8FDF705F9FDF762
:105340003BF9FDF74DF8C820FCF77EFEF04D20201C
:10535000A861FFF72FFFFFF7A1FB4FF0A042906875
:1053600040F00040906090680028FCDBD2F8080113
:1053700040F00040C2F80801D2F808010028FBDB29
:10538000D06820F47C60D060D06840F48070D06039
:10539000D06840F48060D060906840F00100906078
:1053A000C820FFF7AFFBD2F8080140F00100C2F8B7
:1053B0000801C820FFF7A6FB906840F00400906049
:1053C000D4480068D34940F001000860086840F400
:1053D00080300860D048016841F001010160CF4889
:1053E000016821F002010160C16841F00101C16062
:1053F000CA4A1832116841F060011160C749203172
:105400000A6842F001020A60011D0A6822F0700277
:105410000A600A6842F030020A60C04A64213432ED
:105420001160026842F0010202600005026822F089
:1054300002020260C26842F00102C260026842F0E9
:1054400001020260B648026822F002020260C268ED
:1054500042F00102C260B34C206A40F001002062B9
:105460006163206840F001002060C820FCF7ECFD7B
:105470000020FDF7D5F9AC4F4FF40068FF280ED09F
:1054800021152846FCF7D8FBC0B941462846FCF751
:10549000D3FB98B9A1142846FCF7CEFB70B97E72F5
:1054A0000020FDF73BFD787A401CC0B278720428DA
:1054B000F6D39D487E720930FDF7A4FD9B48007825
:1054C0007872032801D903207872FFF7BFFE97F89E
:1054D000320000EBC00101EB00109249486301204B
:1054E00087F8270087F82660F87EB14601284FF438
:1054F000804072D0A8614FF090400821C0F8181089
:105500004FF4FA763046FCF79FFDFFF7C7FA88A103
:105510008948FAF7DFFE052188A20120FFF7B6FBD4
:1055200040F6B830FFF754FA152185A20220FFF7A4
:10553000ADFBB000FFF74CFA252182A20120FFF756
:10554000A5FB7000FFF744FA35217FA20220FFF788
:105550009DFB6420FCF778FD42217CA20120FFF72F
:1055600095FB40F2DC542046FFF732FA3220FCF77C
:105570006BFD2046FFF72CFA77A27AA16E48FAF766
:10558000A9FE6D4A41210320FFF74AFB0120FDF7E8
:1055900047F987F836003046FCF756FD00241C21F9
:1055A0002046FFF7D7FC641CE4B2802CF7D3787850
:1055B00097F82C1000EB41006B4951F820206BA1AB
:1055C0005D48FAF787FE5C4A19210520FFF75EFB6C
:1055D000F87E01280DD016E0FFE7A8624FF0904159
:1055E000082088626420FCF72FFDB87E02F018FEC8
:1055F00086E7BA7E5EA15048FAF76CFE4E4A0F214C
:105600000720FFF743FB4FF4FA70FCF71DFD464BF4
:105610000C208033B8779868FFF78AFCD9688842F5
:105620000ED1FCF70FF801463F4880308068814278
:1056300006D1042087F83D00022087F83C001FE0D7
:10564000042087F83D00012087F83C00FFF7B2FDF9
:10565000FFF724FA4AA13848FAF73CFE364A1821E7
:105660000120FFF713FB49A13348FAF733FE324A12
:105670000A210320FFF70AFB4FF4FA60FCF7E4FC71
:10568000F87C55281DD097F83C0002281DD1FCF766
:10569000B1F897F87010484300F00700062810D1C1
:1056A000FFF7FCF93DA12448FAF714FE224A0A212B
:1056B0000320FFF7EBFA41F28830FCF7C5FC20200D
:1056C000A86297F83C00022806D097F82E0014280C
:1056D00002D9142087F82E00002630464FF00061D2
:1056E0000958001D0E44B0F5E04FF7D3B86C864260
:1056F0007ED0FFF7D3F96420FFF76AF92BA10E489B
:10570000FAF7E8FD0A210C4A032057E00030004078
:10571000000400480074004000980040000400406D
:1057200000100040004401400000002000DC0008A0
:105730004B504F542D0000003C0200204B00000055
:10574000500000004F000000540000002053544D52
:105750005F46336420000000762E31302F30372F23
:105760003236000025732000EC0100202573000074
:10577000464D202D202564206D487A200000000031
:105780002A2A2A44454D4F2A2A2A00007261646958
:105790006F646F6D40692E7561000000204B4559A4
:1057A000204552524F5221200000000020474C4F0C
:1057B00042414C204552524F52212000FFF766FAD9
:1057C0004FF47A70FCF740FC4FF480512846FCF708
:1057D00033FA80B941462846FCF72EFA58B93246CA
:1057E000FDA1FE48FAF776FD2321FC4A062000E0E1
:1057F00002E0FFF715FAFEE74FF40061F848FCF706
:105800001BFA40B9DFF8D8834FF480663146404632
:10581000FCF712FA30B14FF40051F148FCF70CFAE2
:1058200060B3BEE0FF2078710F2087F826000120CA
:10583000B871FFF733F9EBA1E848FAF74BFD012106
:10584000E64A0846FFF722FAFDF73EFBEA4D2861DB
:1058500040F6B830FFF7BCF8FDF736FB28614FF48F
:10586000FA60FFF7B5F8FDF72FFB28614546314692
:105870002846FCF7E1F90028F9D0FBE0012087F881
:105880002200FFF70BF90A2087F83A00FCF7E4FF43
:1058900040F6E4456420FCF7D7FBDFF8608340F274
:1058A000F31600BFC8F800601420FCF7CDFB386F7A
:1058B000A84201D205468246761F722EF2DC97F886
:1058C0002D00A0EBC00000EB80010AEB810A00264E
:1058D0006420FCF7B9FBDFF8288340F2F3154FF0A2
:1058E0001F0BC64805602820FCF7AEFB386FB0429E
:1058F00004D9B0FBFBF1064603950191A0EB0A0128
:1059000097F82D00C0EB0010B1FBF0F03C2800D957
:105910003C20A5F2F3114A42C1B202EBD2706FF003
:105920003F0202EB600040B2FCF7ACFF3B6F691C2A
:10593000B3FBFBF098FBF1F20090B2A1A748FAF795
:10594000C9FCA64A02210120FFF76AF96D1E722DDB
:10595000C7DA0398B0A1401C98FBF0F301980090BF
:1059600097F82D209D48FAF7B5FC9C4A02210120AA
:10597000FFF756F9AD494AF6AA2008604E144FF4D5
:105980008068974D05E041462846FCF755F9002808
:105990009DD031462846FCF74FF90028F3D1FFF798
:1059A00055FC4FF480518E48FCF746F9E8BB4FF4A4
:1059B000FA70FFF70DF8FFF771F8FBF71BFFDFF840
:1059C00038829A4D834608F1800840F6E4464AF64C
:1059D000AA2AC820FCF738FBC5F800A0386FB042EF
:1059E00000D93E675B4692A17C48D8F81420FAF7AC
:1059F00071FC7A4A03210120FFF748F990A177480A
:105A00003A6FFAF767FC754A03210420FFF78EF816
:105A10008CA17248FAF75EFC704A64210720FFF7F8
:105A200035F94FF400516E4800E007E0FCF704F947
:105A30000028CED14FF4C870FEF7CAFF6420FCF7EF
:105A400003FBFBF7D7FE052814DAFFF727F87EA142
:105A50006248FAF73FFC614A14210320FFF716F968
:105A60003220FEF7B5FF3C20FEF7B2FF4FF47A700C
:105A7000FCF7EAFA4FF0010BBA463D4687F820B032
:105A80004FF47A70FCF7E0FAFFF708F895F83C005D
:105A9000401D2877FDF718FADFF85C814546C8F805
:105AA00010006420FCF7D0FAFDF70EFA286164209C
:105AB000FCF7CAFAFDF708FA9FED678B9FED689B2C
:105AC00028619AF82E005546C0F11E008AF82F0072
:105AD000D8ED0A0A4746C8ED100A98ED0B0A88ED82
:105AE000120A9AF83400002874D0A86D03F06CFCF8
:105AF00041EC100BFDF7E8FFB0EE40AAF0EE60AA13
:105B0000B86C03F076F953EC1A2B03F09DF941ECD5
:105B10001A0BA86D03F058FC41EC100BFDF78CFD3F
:105B2000B0EE40BAF0EE60BA386C03F062F953ECB4
:105B30001B2B03F089F953EC1A2B02F0B5FE03F08E
:105B4000FBF8B865A86D03F03FFC41EC100BFDF7C6
:105B5000BBFFB0EE40AAF0EE60AA386C03F049F942
:105B600053EC1A2B03F070F941EC1B0BA86D03F0FA
:105B70002BFC41EC100BFDF75FFDB0EE40AAF0EE00
:105B800060AAB86C03F035F953EC1A2B03F05CF9FA
:105B900053EC1B2B03F02EFB03F0CEF8F8653866B0
:105BA00095F82C00042816D0134964208031086031
:105BB000386EC01C03F01DF941EC100BFDF7A0FD81
:105BC00051EC100B03F0B8F8F866002801DAC7F8BA
:105BD0006C9049E06EE07EE0256C64003C020020A1
:105BE00000040048466163746F72792073657474B1
:105BF000696E677300000000800000202C040040E4
:105C0000C0C62D002564487A2025646D42204B557E
:105C10003D25642020000000472564204D41583D6B
:105C20002564487A204B553D256420000030004013
:105C30002564487A202A2025646D41200000000058
:105C400025642F006D562000205475726E20636FFE
:105C5000696C212000000000000000000000F03FFF
:105C60006666666666A64C40386EC11700EB91709A
:105C700086104AF2104086420DDD0621C320FEF751
:105C80008DFE49F64040FEF73DFF0621C320FEF79A
:105C900085FE85F8359095F94400F96EB8460844BC
:105CA000C1B285F8231095F83520012A18D04FF499
:105CB000967073E0B8EEC01AF8EEE01A95ED162A69
:105CC00001EEC21ABDEEC11A87ED181AC7ED160A09
:105CD00087ED170A64E7386C4110FE48016067E7FA
:105CE00085F8359095F82720012A5AD0022A7CD0D1
:105CF000491CC9B24FF4FA70FEF750FE95F82F1008
:105D0000D8F860004246884270DDF24F3B68B3EB42
:105D1000410FF9DDB0F5AF7F01DD85F815B085F8ED
:105D2000289095F82900401CC0B285F82900322837
:105D300001D985F820B0D8F85810D8F84400091ACD
:105D4000C8F85810D8F85C20D8F84C00101A00EEAB
:105D5000100AC8F85C00F8EEC00A00EE101AB8EE9F
:105D6000C00A02F00FFC40B22873796801447960E0
:105D7000D8F86010029A914202DDA873FE60029189
:105D8000A87B2874287395F8380095F82920801C82
:105D9000824205D9084602F0BBFA6420FEF7B2FE43
:105DA00065E195F82F00D8F86020411C47468A42EB
:105DB00055DDC8490968814251DD85F82A9085F88A
:105DC000289095F82900401CC0B285F829001428B5
:105DD00001D985F820B0B96D786C081AB865FA6CED
:105DE000F96D891A00EE101A01E0C8E014E1F8EE2E
:105DF000C00A00EE100AF965B8EEC00A02F0C2FB54
:105E000040B228736874396E029A914203DDB14A38
:105E1000A873D660029195F91020904200DAE873D9
:105E2000E87B287495F90E00287395F8362085F8DC
:105E3000372095F82420012A0ED932290CDD95F956
:105E40004310082908DD0A2806DD4FF4FA60FEF742
:105E5000DFFD85F843900AE102F05CF907E10020DC
:105E600002906420E87395F82800401C85F828000B
:105E700085F82990B86D7864F86DF86495F8240079
:105E8000022876D995F82A00401C85F82A0095F852
:105E90003400E0B3A86D03F097FA41EC100BFDF766
:105EA00013FEB0EE40AAF0EE60AA386B02F0A1FF3C
:105EB00053EC1A2B02F0C8FF41EC1A0BA86D03F04B
:105EC00083FA41EC100BFDF7B7FBB0EE40BAF0EEF1
:105ED00060BA786B02F08DFF53EC1B2B02F0B4FF1D
:105EE00053EC1A2B03F086F902F026FF7866C01CEB
:105EF00002F07FFF41EC100BFDF702FC9FED761BDB
:105F000051EC100B53EC112B02F082FD00E01CE071
:105F100002F012FF3867D7E91921531A032293FBC5
:105F2000F2F211447966B96695F82F20914220DD8E
:105F300095F82A1005291CD995F844100844C1B2D7
:105F40004FF4FA70FEF72AFD91E097ED0D0AD7EDB8
:105F50000C0A95ED161AB8EEC00AF8EEE00A00EE4B
:105F6000C10ABDEEC00A87ED190A10EE100ABEE79D
:105F7000FFE75B48016821F00101016077E095F8D7
:105F80002F10D8F8602047468A422EDD514A126809
:105F9000B2EB410F29DD85F8289095F82910491CAE
:105FA000C9B285F8291095F83820921C91420FD972
:105FB000C1B24FF4FA70FEF7F1FC97ED120AF8EE59
:105FC000C00A97ED100AB8EEC00A02F0DBFA287397
:105FD000386E0299884204DD297BA9733D49CE6061
:105FE0000290A87B2874287341E03D48016821F0A5
:105FF00001010160386B7864786BC8F84C00354952
:1060000000200290C1F80C9085F8299095F828009E
:10601000401C85F828002AE0906D50642D4FD06D0B
:10602000C8F84C00C7F80C90CDF8089095F82800F7
:106030004E46401C85F82800687D012813D195F84C
:1060400029000A280FD9796891FBF0F20A2A02DDAB
:106050004FF4FA6005E091FBF0F010F1140F02DA52
:10606000C820FEF7D5FC7E606E7585F8296095F82E
:106070002810FA2917D0002095F82920FA2A14D0E0
:10608000002210430CD0134AC2F80C9085F80D90F2
:1060900085F80C9085F8119085F820B085F843902C
:1060A000C22904D005E00120E6E70122E9E7FEF776
:1060B000DDFC95F82800FA2801D1FEF709FD687982
:1060C0004646002898F804000CD000F01F00032872
:1060D0007ED0ADE100010020000000000000F83F8C
:1060E00000100040C0B285F83F0000F00F0185F8B5
:1060F00040100A2802D1FCF7E7FE3061B0884FF06B
:106100001651B046B1EB005F03D1FEF7E1FC85F814
:10611000119095F84000012874D1FF4895F90C6062
:10612000C068C01C02F065FE41EC100BFDF7E8FAF8
:1061300053EC182B51EC100B03F05CF802F0FCFD53
:106140000746F548C1680161D8F86000322859DD7A
:1061500096FBF7F000EBD0706E73401085F84300AB
:1061600095F90E0095F91010401AC01C02F041FE7E
:1061700041EC100BFDF7C4FA51EC100B02F0DCFD02
:1061800095F94310552E91FBF0F040B285F843008D
:1061900003DC95F91010002904DA00EBD0704010F0
:1061A00085F8430095F83B0000F134018E4209DB8D
:1061B0004030864206DC95F9430000EBD070401079
:1061C00085F84300002F05DB95F94300002800E027
:1061D0002BE102DA85F8439004E00A2802DD0A2068
:1061E00085F8430095F9430095F90B10401A00EB30
:1061F000D07001EB600085F84300E872FE4201D1E7
:1062000085F8439095F8400002280CD1FBF7E2FA9C
:10621000C2A253210420FEF703FD95F84300800637
:10622000000EFBF7C5FA95F8400003280BD195F84E
:106230002D20BBA1BD482B6FFAF74CF8BB4A3A2181
:106240000320FEF7EDFC287F07280DD0B8A1B74842
:10625000FAF740F8B54A55210720FEF7E1FCB34AAA
:1062600014210720FEF7DCFC95F84000042827D114
:10627000D8F810100A20B1FBF0F200FB1212B1FBAB
:10628000F0F0CDE9000295F8383095F82E20AAA15B
:10629000A648FAF71FF8A54A3A210120FEF7C0FCEC
:1062A0009D48AAA1406900906A7A95F82B309F48D2
:1062B000521CFAF70FF89D4A3A210220FEF7B0FC73
:1062C00095F8400005280AD1686D20B3A2A197482F
:1062D000FAF700F8954A70210320FEF7A1FC95F823
:1062E000400006281AD195F84100042816D095F9E7
:1062F0000D20002A00DA524299A18C48F9F7EAFFF2
:1063000095F90D00894A00284FF002014FF0010075
:1063100002DBFEF70BFC01E0FEF744FC95F83F00C2
:1063200032280BD195F8340088B18FA17F48F9F756
:10633000D1FF7E4A3A210420FEF772FC95F827002F
:10634000012806D095F840000B2853D054E088A1CE
:10635000ECE795F84100012804D0022816D0032864
:1063600017D036E095F84000072836D16A49086909
:10637000C01000D540420861172801DD17200861D0
:10638000097C95F9110001F077FF49E002F072F9FC
:106390001FE0D8F86020032198ED120A92FBF1F17A
:1063A000F8EEC00A98ED100ACEB2B8EEC00A02F0BC
:1063B000E9F8C0EBC0010A2091FBF0F040B2314691
:1063C000FCF77CFA40210820FEF778FFAA2002F0B3
:1063D000BDF895F8410004280BD006244021204642
:1063E000FEF76CFFAA2002F0B1F8641CE4B2082C9E
:1063F000F4D3DAE3FEF76CFBD8F86C00002802DD7A
:10640000C0B2FCF7C1F995F8270002280BD05AA1B9
:106410004648F9F75FFF454A02210620FEF736FCA1
:1064200040212046D0E756A1F2E7FBF7E3F9687672
:10643000A87920B101286DD002286CD0B5E3364E82
:106440006878843656F82020AFF6E0413748F9F7EF
:1064500041FF364C354A17340A216078FEF716FCA6
:1064600095F8362047A13148F9F734FF60782F4A74
:106470005F21FEF70BFC687806EB8000AFF6145145
:1064800082682A48F9F726FFA078284A0A21FEF7F1
:10649000FDFB95F824203BA12448F9F71BFFA078C9
:1064A000224A5F21FEF7F2FB687806EB8000AFF628
:1064B000445102691D48F9F70DFFE0781B4A0A2193
:1064C000FEF7E4FB95F94420012A01DA2FA100E050
:1064D00030A11648F9F7FEFEE078144A5821FEF77D
:1064E000D5FB687806EB8000AFF6805182690F48D3
:1064F000F9F7F0FE20790D4A0A21FEF7C7FB95F85F
:10650000300027A1C0F106020848F9F7E3FE207920
:10651000064A49E064E1A4E20001002052000000C4
:106520004725643C25646D563E2000003C02002057
:1065300044454D4F00000000532530326420204672
:1065400025642520206476256400000050256428F9
:106550002564292564487A00432E422E000000005D
:1065600025303264000000004742462E0000000043
:106570004742562E00000000446570746800000019
:1065800050696E002D202564200000002D28256410
:10659000292020002D282B25642920200000000020
:1065A0002D202564202000005F21FEF76FFB687816
:1065B00006EB8000AFF64C61026AF948F9F78AFEF3
:1065C0006079F74A0A21FEF761FBF64995F8390030
:1065D0000A5CAFF23401F248F9F77CFE6079F04AC8
:1065E0005F21FEF753FB687806EB8000AFF684610D
:1065F000826AEB48F9F76EFEA079E94A0A21FEF7B4
:1066000045FB6B7E95F83A20E7A1E548F9F762FE75
:10661000A079E34A3121FEF739FB687806EB800068
:10662000AFF6B861026BDE48F9F754FEE079DC4A58
:106630000A21FEF72BFB95F82B20AFF29C01D848DE
:10664000F9F748FEE079D64A6021FEF71FFB68782B
:1066500006EB8000AFF6EC61826BD148F9F73AFEA9
:10666000207ACF4A0A21FEF711FB687895F82C10A2
:1066700000EB4100CB49D03151F82020AFF6147126
:10668000C748F9F727FE207AC54A3221FEF7FEFAFD
:10669000687806EB8000AFF62C71026CC048F9F701
:1066A00019FE607ABE4A0A21FEF7F0FA95F8322008
:1066B000AFF21411BA48F9F70DFE607AB84A5F21BB
:1066C000FEF7E4FA687806EB8000AFF66071826C42
:1066D000B348F9F7FFFDA07AB14A0A21FEF7D6FACE
:1066E00095F84120AFF26411AD48F9F7F3FDA07AB7
:1066F000AB4A5F21FEF7CAFA687806EB8000AFF676
:106700009471026DA648F9F7E5FDE07AA44A0A21E2
:10671000FEF7BCFA6A7FAFF29411A148F9F7DAFDEF
:10672000E07A9F4A5F21FEF7B1FA687806EB8000B5
:10673000AFF6C871826D9A48F9F7CCFD207B984A74
:106740000A21FEF7A3FA95F83100C0F10902AFF271
:10675000B0119348F9F7BEFD207B914A5F21FEF707
:1067600095FAAA7E93A18E48F9F7B4FD607B8C4A16
:106770000A21FEF78BFAE87E78B392A18848F9F7F0
:10678000A9FD607B864A1E21FEF780FA68788FA1FA
:1067900006EB8000026E8248F9F79CFDA07B804AE0
:1067A0000A21FEF773FA012487A201212046FEF791
:1067B0006DFAA41CE4B2082CF6D395F82600FF214C
:1067C00001EB4001E977042801D90720E87780A28E
:1067D0000121E87FFEF75AFAE7E1FFE77DA1CDE767
:1067E00095F826000E38E877706800F00701012957
:1067F00002D1FAF7FFFF68766A4C6878303473A1EB
:1068000054F820206648F9F765FD654A0A21012001
:10681000FEF706FA6A7A71A16148521CF9F75AFD2F
:106820005F4A4B210120FEF7FBF9687867A104EB72
:10683000800082685A48F9F74DFD594A0A21022022
:10684000FEF7EEF931690A20B1FBF0F200FB1213FA
:10685000B1FBF0F263A15248F9F73CFD504A4B21DD
:106860000220FEF7DDF9687858A104EB8000026988
:106870004B48F9F72FFD4A4A0A210320FEF7D0F9C9
:1068800095F82D20AFF204314548F9F723FD444A2D
:106890004B210320FEF7C4F968784CA104EB80007B
:1068A00082693F48F9F716FD3D4A0A210420FEF7A8
:1068B000B7F9A4F14C006A7E43694DA13848F9F755
:1068C00009FD374A2D210420FEF7AAF968783FA177
:1068D00004EB8000026A3248F9F7FCFC304A0A21D6
:1068E0000520FEF79DF946A12D48726FF9F7F2FCDD
:1068F0002B4A4B210520FEF793F9687833A104EB6E
:106900008000826A2648F9F7E5FC254A0A2106201C
:10691000FEF786F968782DA104EB8000026B204811
:10692000F9F7D8FC1E4A0A210720FEF779F995F8F5
:10693000340098B335A11A48F9F7CCFC184A4B211A
:106940000720FEF76DF9687820A104EB8000026B48
:106950001348F9F7BFFC124A0A210720FEF760F935
:10696000287F072862D02BA10D48F9F7B3FC0C4A09
:106970000A210820FEF754F9012413A20121204620
:10698000FEF74EF9641CE4B2092CF6D395F8260004
:1069900012284DD00021132854D04AE044E045E0AD
:1069A0003C0200201C01002028256429202D2025E0
:1069B00064202000464D20202020202D2025646DBD
:1069C000487A2000284F4E2920000000257300003F
:1069D0003E000000284F4646290000002D20256477
:1069E000000000002D2025642E25642056000000A4
:1069F000282564292D202564487A202000000000E5
:106A00002D20256420677220200000002D204742A1
:106A100046200000456E747279204B455920202095
:106A20002D2C2B2000000000FDA184E7FEA19BE798
:106A3000012100221143162806D00020014305D071
:106A4000FCA205E00122F5E70120F7E7AFF28002A2
:106A50000121E87FFEF7E4F84FF6E850FEF752F820
:106A6000A3E095F83C00022865D0FCF7F9FAF2485B
:106A700090F80014801E90F8000441EA0020B060F5
:106A8000EEA1F048F9F726FC0121EE4A0846FEF790
:106A9000FDF8B268ECA102F50053EA48F9F71AFCD8
:106AA000E84A59210120FEF7F1F895F91220E8A1F2
:106AB000E448F368F9F70EFCE24A02210320FEF7EE
:106AC000E5F8307900F00300022810D9E4A1DD4890
:106AD000F9F700FCA87FFA2101EBC000C1B2D94A46
:106AE0000320FEF7D3F84FF49670FBF7ADFA0024BD
:106AF0002B212046FEF72EFA641CE4B27F2CF7D33C
:106B0000D84AD9A1CF48F9F7E5FBCE4A02210520A2
:106B1000FEF786F8D8A1CB48F9F7DCFBC94A052176
:106B20000720FEF77DF8DAA1C648F9F7D3FB052167
:106B3000C44A08208EE7FDF7B1FFDAA1C148F9F792
:106B4000C9FBC04A05210220FEF7A0F8C54ABD488E
:106B500002F10C01F9F7BEFBBA4A1E210420FEF730
:106B60005FF8D4A1B748B268F9F7B4FBB54A1D2164
:106B70000620FEF755F895F91300009095F91230AC
:106B8000CFA1B048F268F9F7A5FBAE4A1D21072056
:106B9000FEF746F841F28830FBF756FAFDF77EFF24
:106BA00085F806B0152085F82600AA4685F81490C9
:106BB0004FF40051C748FBF73FF8A8B1C54D4FF45B
:106BC000805631462846FBF737F8D8B3B1102F4628
:106BD0002846FBF731F8002876D071103846FBF7CD
:106BE0002BF8002871D00CE3BB48016821F00101AB
:106BF000016055469AF82600FBF730FD85F80890AD
:106C0000E8784E46012826D04FEA08074FF4005195
:106C1000B048FBF711F888B3687980B3A8790128E8
:106C20007ED002287CD095F82600401CC0B285F8A2
:106C300026000E2802D9584685F826B0C0B2FBF7C8
:106C40000DFD00E075E095F826000F2800D22871B0
:106C500040F6C410FEE340F6B830FDF7B9FE9D4F94
:106C60004FF400513846FAF7E7FF0028F8D0C82063
:106C700085F8290085F82800EE70ECE300E02BE0B1
:106C80002320FBF7E1F9287D401CC0B22875396844
:106C90008842BBD96879C0436871FDF7FFFE85F86B
:106CA00003B0AE72687988B1287985F82600FAF7C2
:106CB000A1FD687695F82600FBF7D0FCAE714FF485
:106CC000FA60FDF785FEE0E2FDE3FDE385F826606E
:106CD000C820FBF7B9F9F1E7FDF7E0FE40F2DC5020
:106CE000FDF776FE95F82700401CC0B285F8270016
:106CF000032801D985F827B0FBF75EFD82202872B2
:106D000085F820B0C820FBF79FF9F02085F829000E
:106D100085F828009CE703E0162085F8260097E711
:106D200095F82600401CC0B285F826001628F3D836
:106D300087E76949086820F0010008609AF8260092
:106D40000C2869D009DC0C28BDD2DFE800F01F65F3
:106D50006565656565656565656512285DD008DCF6
:106D6000A0F10D010529AED2DFE801F0F05656562C
:106D700056001528E5D004DC13284FD01428A2D1E2
:106D8000FEE31628DDD04D289DD1FAE3FDF786FEFF
:106D90006420FBF759F98AF807B09AF81C00072815
:106DA00020D04EA12748F9F795FA264A1E21022045
:106DB000FDF76CFF4FF44870FDF70AFE4FF4617069
:106DC000FDF706FE4FF47A70FBF73EF911E223203F
:106DD000FBF73AF9287D401CC1B229753868814219
:106DE00002D907E04746554631463A48FAF724FFAC
:106DF0000028ECD0287D3968884210D93220FBF772
:106E000023F997ED0D0AF8EEC00A97ED0C0AB8EEDB
:106E1000C00A01F0FFFB67E0F4E17EE2FFE289E1F6
:106E20002D204742562000004B4559204F4B212032
:106E3000202000006F00000005D00008436F64654B
:106E4000202D3E003C02002025582558000000005F
:106E5000456E742E4B65793C25643E2025303458B0
:106E600020000000585700083C53544D333246333D
:106E7000643E2025732000006D61696C3A207261C8
:106E800064696F646F6D40692E7561202000000099
:106E9000687474703A20726164696F646F6D2E6FEC
:106EA000726700002020204B455920204F4B2021A5
:106EB000200000004B6F64653A20253034582000D4
:106EC0004B65793A202025303458202825642D251B
:106ED0007829000000040048001000402A204445A2
:106EE0004D4F202A000000002873396B786B49430E
:106EF00000FB001001F07DFF41EC100BFCF748FE99
:106F000051EC100B01F018FF801001F072FF41EC02
:106F1000100BFCF7F5FB51EC100B01F03DFFC4B278
:106F20000C2C00D90C2495F8340080B1FBA1FE484C
:106F3000F9F7D0F90121FC4A0846FDF7A7FE95F9BB
:106F40000C0010F15A0F04DA012103E0B3E1F7A1BC
:106F5000EDE7002110F13C0F01DD012000E00020F1
:106F6000014313D0F4A1F048F9F7B4F9EE4A5321E4
:106F70000120FDF78BFE4FF49670FDF729FDC82028
:106F8000FDF726FDBE20FDF723FD41E0092C01D9C8
:106F9000032002E0062C03D9022085F8380001E026
:106FA00085F838B0E6A1E048F9F794F9DE4A5321B4
:106FB0000120FDF76BFE4FF49670FDF709FD4FF4CD
:106FC000C870FBF741F84FF41670FDF701FD4FF460
:106FD000FA70FDF7FDFC95F90C0001F00AFF53EC87
:106FE000192B01F015FD41EC100BFCF711FE53ECD1
:106FF000102B51EC180B01F00BFD01F023FCA865E0
:1070000095F8340008B1287B01E06FF05900287032
:10701000CCA1C548F9F75EF9C34A02210620FDF765
:10702000FFFD4FF44870FDF7D3FCCC4E4AF6AA277B
:1070300078E000BF95F83800009095F90C302246B2
:10704000C7A1B948F9F746F9B74A01210420FDF76D
:107050001DFEA86D02F0B8F941EC100BC5A153EC70
:10706000102BB148F9F736F9AF4A1E210820FDF779
:10707000D7FD4FF480613046FAF7DEFD18BB287B60
:10708000401C28734FF4FA70FDF7A2FC95F90C0030
:1070900001F0AFFE53EC192B01F0BAFC41EC100BE0
:1070A000FCF7B6FD53EC102B51EC180B01F0B0FCC3
:1070B00001F0C8FBA86595F8340008B1287B01E011
:1070C0006FF0590028704FF400613046FAF7B4FDB4
:1070D00018BB287B401E28734FF41670FDF778FC10
:1070E00095F90C0001F085FE53EC192B01F090FC92
:1070F00041EC100BFCF78CFD53EC102B51EC180BF2
:1071000001F086FC01F09EFBA86595F8340008B1FB
:10711000287B01E06FF0590028706420FAF794FF93
:10712000974807604FF480513046FAF785FD0028F4
:1071300080D05EE028462F6F00F8149FAA4680F8A2
:10714000159080F8149085F820B040F6E445AF42E1
:1071500000DD2F463A468BA17348F9F7BBF8724A17
:107160000A210320FDF792FD4FF47A70FDF730FC01
:10717000C82F3EDD88A16C48F9F7ACF86A4A0521B2
:107180000720FDF74DFD0220FAF75EFF734F5646CC
:1071900029E000BF4EF66020FDF7B4FC4FF400512B
:1071A0003846FAF749FDF0B94FF4FA60FDF710FCE4
:1071B0000020FDF759FB4FF47A70FDF709FC42F20D
:1071C0001070FDF79FFC326FAA4200DD2A466DA1C8
:1071D0005548F9F77FF8544A0A210320FDF756FD78
:1071E0001420FAF731FF307D401CC0B230751E28E4
:1071F000D0D38AF807904FF4FA70FAF725FFFDF71D
:107200004DFC7FE1401E10F0FF0055468AF8260035
:1072100006D00F2800D22871A879012804D00AE0EE
:107220000E2085F82600F6E795F826000E2802D1F4
:10723000162085F8260040F6C410FDF7C9FB95F826
:107240002600FBF70BFAC82060E21420FAF7FCFED8
:10725000287D401CC0B22875316888422ED940F67E
:10726000B830FDF7B5FBE87E90B185F81B904FF480
:107270008040B8614FF09041082088614FF4FA6077
:10728000FDF7A6FB6420FAF7DFFE8AF820B0DFE402
:1072900085F81BB04FF48040B8624FF09041082051
:1072A00088623220FAF7D0FEA87E00F0B9FF3220C3
:1072B000FAF7CAFEE2E72F46464655464FF480519C
:1072C0003846FAF7B9FC0028BFD015F8260F401E43
:1072D000C0B22870FBF7C2F9BAE41920FAF7B4FE7D
:1072E0009AF81410491CC9B28AF81410D8F8002072
:1072F00091427CD900268AF822B001F0EDF972277C
:1073000040F2F3152A4805601920FAF79DFEFAF7B6
:1073100071FAB04250DD06464CE068E04772617594
:107320006E642042462D00003C02002047726175C9
:107330006E642042562D00004572726F722100006B
:107340004F4B2000416D706C69742E205068617342
:1073500065202046696C747200000000000400483B
:107360003C253032643E203C25643E203C4625646A
:107370003E200000203C25302E33663E20200000B9
:10738000003000402A2A2A202564206D56202A2A0F
:107390002A20202020000000436F696C20626C2EA0
:1073A000707265737320274D656E752700000000AD
:1073B0002C040040CAF86C50FE4890FBF5F1C81749
:1073C00001EBD0604211FCA1FE48F8F783FFFD4AB3
:1073D00010210520FDF75AFC6D1EBD4292DCFBF723
:1073E000EBF94FF4FA60FDF7F3FAFDF757FB4FF4B2
:1073F0008051F548FAF720FC00283FF46EAF9AF868
:107400002210504600297DD190F82610491E8AF896
:10741000261000BF40F6C410FDF7DAFA13E708683B
:1074200020F00100086045465746B3E01920FAF7FE
:107430000BFE387D401CC0B23875296888427DD962
:10744000FDF72CFB87F822B007F807BF5C46C5F8AC
:10745000749001E046E108E2FBF7F2F97C76DBA1EB
:10746000D848F8F737FFD74A0A210320FDF70EFC6A
:1074700040F6B8363046FDF7ABFA7C762868FF1F39
:10748000C0EB00108000FAF7DFFDD3A1CD48F8F77C
:1074900021FFCC4A0A210320FDF7F8FB3046FDF717
:1074A00097FA2868C0EB00108000FAF7CDFD00269F
:1074B0004FEA060495ED0D0AF8EEC00A95ED0C0AA8
:1074C000B8EEC00A01E024E14FE301F0A3F806445E
:1074D000C820FAF7B9FD641CE4B2082CEAD3F0170F
:1074E00006EB5070C0105A3040426867B0F5B47F68
:1074F00002DDA0F5B4706867002802DA00F5B47008
:10750000686700E0F8E3401C6867FBF799F987F8C3
:1075100020B0286832214843FAF796FD95ED0D0A10
:10752000F8EEC00A95ED0C0AB8EEC00A01F072F848
:10753000002800DA4042582812DA00E02AE0AAA126
:10754000A048F8F7C7FE9F4A0A210520FDF79EFBD9
:10755000C820FDF73DFA9620FDF73AFA64200EE0C8
:10756000A3A19848F8F7B6FE964A0A210520FDF730
:107570008DFB4FF4FA60FDF72BFA40F6C41001E0E2
:1075800022E031E0FDF724FA4FF47A70FAF75CFD5F
:10759000FDF784FA4FF480518B48FAF74DFB002831
:1075A0003FF444AF97F8220058B997F82600401EE0
:1075B00087F8260040F6C410FDF70AFAC820FAF74B
:1075C00043FD87F8079097E3401E8AF8260021E7DD
:1075D0002820FAF739FD387D401CC1B23975D8F83A
:1075E0000000814201D907E057464FF480512846F8
:1075F000FAF722FB0028EBD0387DD8F80010464679
:10760000884253D9B068FDF793FCF16888421DD1D8
:10761000FAF718F8B168884218D177A16948F8F7E5
:1076200059FE684A1E210320FDF730FB4FF4FA7023
:10763000FDF7CEF94FF47A70FDF7CAF9B0897149B8
:10764000020A0A7188715520F8741DE06EA15D4828
:10765000F8F740FE5B4A00210120FDF717FB6FA100
:107660005848F8F737FE574A00210320FDF70EFB74
:107670006420FDF7ADF95020FDF7AAF96420FDF76D
:10768000A7F9B87C401CB8744FF4805631462846A0
:10769000FAF7D2FA0028F9D00120FBF793FC4FF457
:1076A000FA60FAF7D1FC2020A86225E397F91200CE
:1076B00005281ADA5348B97FD538014411F80C2D42
:1076C000521C02F00F020A70C178027841EA0231BE
:1076D00042788078120242EA001001434FF4487069
:1076E000C8F80C10FDF774F906E351A13548F8F716
:1076F000F1FD344A00210320FDF7C8FA6420FDF7AC
:1077000067F95020FDF764F94FF4FA60FAF79CFC32
:10771000F8E34C4E306820F0010030609AF8260003
:1077200055460C2842D009DC0C2840D2DFE800F096
:10773000A4C1CDD9EFFFECEBEAE9E8E7122837D096
:1077400008DCA0F10D00052831D2DFE800F0EFEEF3
:10775000EDECEB0015282CD004DC132874D0142891
:1077600025D1B8E1162870D04D2820D1EBE11420A6
:10777000FAF76AFC287D401CC1B22975386881423D
:107780007BD985F822B0306820F00100306095F890
:107790002D0001286CD0584685F82DB0C0B2F9F7FD
:1077A0003FFF0021084600F03DFE4FE01BE197E05F
:1077B0007AE1B3E100D8B8052A20256420487A2070
:1077C0002A2020003C02002000040048204E6F20A8
:1077D00046657272697465002054616B6520466568
:1077E0007272697465000000204572726F72210028
:1077F000204F4B2100000000204F4B212020202053
:10780000200000002101002020726164696F646F14
:107810006D40692E7561202020000000202020206E
:10782000204552524F5221202020202020000000CD
:1078300020204552524F5221204E3E3D35202120DE
:10784000200000000010004038E172E14FF47A702F
:10785000FDF7BEF896202872C5F85490C7F804B01A
:1078600085F820B0C820FAF7EFFB4DE305E0FFE70D
:10787000022085F82D0091E747464FF48061F948D2
:10788000FAF7DAF900283FF472AF95F8220038BB16
:10789000287F07280BD01C2095F82E10491CC9B250
:1078A00085F82E1081421BDD85F82E0058E11E2040
:1078B000F2E795F83600401CC0B285F8360019286A
:1078C0000ED9192085F836004AE195F82400401CAD
:1078D000C0B285F82400032802D9032085F82400CB
:1078E0003EE195F84400401C40B285F8440005286C
:1078F00002DD052085F8440095F82D00D1E069E00F
:107900005CE048E039E02CE01DE010E0FFE795F88E
:107910003000401EC0B285F83000FF2801D185F844
:1079200030901DE1B1E098E08CE076E066E095F8FB
:107930003900401CC0B285F83900042802D904205F
:1079400085F839000CE195F83A00401CC0B285F882
:107950003A00142802D9142085F83A00FAF77CFF7F
:10796000FEE095F82B00401CC0B285F82B000A28D9
:1079700002D90A2085F82B00F2E095F82C00401C73
:10798000C0B285F82C00072802D9072085F82C0002
:10799000FBF722FAE4E095F83200401CC0B285F80B
:1079A0003200062802D9062085F83200C1B201EB68
:1079B000C10000EB0110AC494863D1E095F84100EB
:1079C000401CC0B285F84100032802D9032085F885
:1079D0004100C5E0687F401CC0B268775A2801D9D1
:1079E0005A206877BCE095F83100401EC0B285F897
:1079F0003100FF2801D185F83190B1E0E87E0128FF
:107A00000AD1A87E401CC0B2A876652801D965209D
:107A1000A876C0B200F004FCA2E0287F072875D049
:107A2000FDF73CF8AFF64C319048F8F753FC8F4A1D
:107A30001E210320FDF72AF9C820FCF7C9FF4FF4E7
:107A4000C8708BE0687A401CC0B26872032801D904
:107A500003206872FDF7FAFB82E095F83300401EC0
:107A6000C0B285F833001E2802D21E2085F83300EC
:107A7000FBF72AFAC8F81000464647F23050FDF7E7
:107A800041F8FBF721FA30616AE095F82D00401CBF
:107A9000C0B285F82D00022802D9022085F82D00F9
:107AA000C0B2F9F7BDFD5BE0E86E401EE8667228E3
:107AB00001D27220E866FAF77FFE51E0D8F8741020
:107AC000491CC8F87410B1F5B47F01DBC8F8749094
:107AD000FAF7B6FE44E0287F072817D0FCF7DEFF50
:107AE000AFF608416148F8F7F5FB604A1E21032014
:107AF000FDF7CCF8C820FCF76BFF4FF4C870FAF71D
:107B0000A3FA00BFFCF7CAFF2AE0FFE70120FBF75A
:107B100005FA4FF49670FCF75BFF21E095F834000E
:107B2000401CC0B285F83400012819D985F834B05A
:107B300016E00220A8714D2085F826004FF4FA7057
:107B4000FCF746FFDEE7A87F401CC0B2A8770F28ED
:107B500001D90F20A877FCF7A1FF3220FAF774FAB9
:107B6000A87A80BB40F6C410C4E1414F386820F0C9
:107B7000010038609AF8260055460C287AD009DCB6
:107B80000C2858D2DFE800F04258637888949FAC04
:107B9000B9C6D9E412286ED008DCA0F10D00052882
:107BA00049D2DFE800F0EFFEECEBEA00152870D0D8
:107BB00004DC13286ED014283DD152E116286AD077
:107BC0004D2838D185E197E11E20FAF73DFA287D4E
:107BD000401CC0B228753168884218D985F822B097
:107BE0003968584621F00101396095F83810491C70
:107BF000C9B285F83810032901D985F838004FF447
:107C0000C870FCF7E5FE032070607DE146464FF446
:107C100000611448FAF710F80028D5D095F8220032
:107C200048B995F82E00401E10F0FF0085F82E0090
:107C300001D185F82EB059E195F83600401EC0B24A
:107C400085F83600FF2801D185F836904EE195F889
:107C50002400401E10F0FF0085F8240001D185F8B3
:107C600024B043E100040048004401403C020020ED
:107C70000010004075E0DBE095F84400401E40B283
:107C800085F84400002801DA85F8449095F82D0025
:107C9000CBE009E1D8E012E195F83000401CC0B219
:107CA00085F83000062802D9062085F830001DE14D
:107CB00095F83900401E10F0FF0085F8390001D119
:107CC00085F839B012E195F83A00401EC0B285F847
:107CD0003A00FF2801D185F83A90FAF7BDFD05E199
:107CE00095F82B00401EC0B285F82B00032802D265
:107CF000032085F82B00F9E004E195F82C00401EE4
:107D0000C0B285F82C00FF2801D185F82C90FBF734
:107D100063F8EBE095F83200401EC0B285F83200FF
:107D2000FF2802D1484685F83290C1B201EBC1006C
:107D300000EB01109A494863D8E095F84100401ED5
:107D400010F0FF0085F8410001D185F841B0CDE089
:107D5000687F401EC0B26877502801D250206877F3
:107D6000C4E095F83100401CC0B285F83100092804
:107D700002D9092085F83100B8E04AE031E025E079
:107D80000FE0FFE7E87E01280AD1A87E401EC0B2BE
:107D9000A876582801D85920A876C0B200F040FA39
:107DA000A4E0287F072877D0FCF778FEAFF6D461EF
:107DB0007C48F8F78FFA7B4A1E210320FCF766FF08
:107DC000C820FCF705FE4FF4C8708DE0687A401EAD
:107DD000C0B26872FF2801D185F80990FDF736FA24
:107DE00084E095F83300401CC0B285F833005A286F
:107DF00002D95A2085F83300FBF766F8C8F810005E
:107E0000464647F23050FCF77DFEFBF75DF83061E7
:107E10006CE095F82D00401E10F0FF0085F82D0055
:107E200002D1584685F82DB0C0B2F9F7F9FB5DE0F4
:107E3000E86E401CE866B0F5FA7F02D340F2F3101A
:107E4000E866FAF7B9FC51E0D8F87410491EC8F892
:107E5000741003D54FF4B471C8F87410FAF7F0FC3D
:107E600044E0287F072817D0FCF718FEAFF694717E
:107E70004C48F8F72FFA4B4A1E210320FCF706FF67
:107E8000C820FCF7A5FD4FF4C870FAF7DDF800BF75
:107E9000FCF704FE2AE0FFE70120FBF73FF84FF470
:107EA0009670FCF795FD21E095F83400401EC0B2B5
:107EB00085F83400FF2819D185F8349016E00220A7
:107EC000A8714D2085F826004FF4FA70FCF780FD6C
:107ED000DEE7A87F401EC0B2A8770C2801D20C2094
:107EE000A877FCF7DBFD6420FAF7AEF8A87A18B99A
:107EF0004FF4FA60FCF76CFD4FF49670FAF7A4F8B3
:107F000085F820B08AF82290274D4FF4007631464C
:107F10002846F9F791FE28B34FF49670FAF794F8D3
:107F200031462846F9F788FEE0B1FCF7B7FD1FA1FE
:107F30001C48F8F7CFF91B4A26210320FCF7A6FEC0
:107F40004FF44870FCF744FD4FF41670FCF740FD09
:107F50004FF4C870FCF73CFD2020A86241F2883045
:107F6000FAF772F8D8F80410491CC8F80410B1F5F3
:107F7000E04F0FD3C8F80490DAF870004E4655462B
:107F8000B0F57A7F01D285F820B0FCF7A1FD6E73C1
:107F900085F8436007484AF6AA210160FDF791BDC4
:107FA000004401403C020020000400483C204F46B1
:107FB00046203E000030004000B51620FAF730FCA5
:107FC000524A82F8380001202432FAF729FC9074D2
:107FD000D0740220FAF724FC10700320FAF720FC7A
:107FE00050750420FAF71CFC90750520FAF718FC70
:107FF00050720620FAF714FCD0710720FAF710FC33
:1080000010720820FAF70CFC10730920FAF708FC2C
:1080100090730A20FAF704FC50770B20FAF700FC63
:1080200002F8070C1820FAF7FBFB50730C20FAF744
:10803000F7FB82F820000D20FAF7F2FB02F80A0C99
:108040000E20FAF7EDFB90760F20FAF7E9FBD073DC
:108050001220FAF7E5FB03461120FAF7E1FB43EAA9
:1080600000209064243A5A2801D25A20D066142065
:10807000FAF7D6FB254B803398671320FAF7D0FB2D
:1080800018B1986F00F5807098671A20FAF7C8FB4E
:10809000D8671920FAF7C4FB18B1D86F00F58070C3
:1080A000D8671520FAF7BCFB82F82E001F20123289
:1080B000FAF7B6FB82F822001720FAF7B1FB5072EC
:1080C000134890F8000450701148401C90F80004C8
:1080D00010700F48001D90F800040D49891C91F89C
:1080E000001440EA012098600948401D90F80004FF
:1080F0000749C91C91F8001440EA0120D8600448DF
:10810000801D90F80004D07400BD00000000002025
:1081100001D000082DE9F0413E4A012110462DED25
:10812000028B10F8234F92F90C30807D002B27DB57
:10813000517F8B4269DC4FF4C86201280AD00228C3
:108140000BD0032815D004285FD1C3EB03104000E7
:10815000214654E02146104651E0322B03DA2146F5
:108160004FF448704BE04A2BF4DD214640F6FC000A
:1081700045E00A2093FBF0F04FF496714843E7E79F
:10818000244D92F831708035EE6EBE423DDD13F124
:108190004B0F3ADD012800D1022192F82C00032870
:1081A0000CD192F82D002623A3EB40002B6E9842B1
:1081B00004DD4FF4487011FB00F0C9E792F830007D
:1081C000F6EE000A00EE100AB8EE400A20EE200A91
:1081D00010EE100A01F0F8F89FED0F1B53EC112B75
:1081E00000F062FB41EC180B204600F019FE53EC46
:1081F000182B00F00DFC00F0CFFDC1B2BE20BDEC8D
:10820000028BBDE8F041FCF7C9BBBDEC028BBDE8B9
:10821000F081000000000020000000000000E03FAE
:1082200010B54C3800F0FCFD9FED111B53EC112BE9
:1082300000F0EEFB00F0B0FDC4B280210020FAF7A0
:10824000F1FE4FF47A70FCF75DFC31210020FAF763
:10825000E9FEB9210220FAF7E5FE4B211020FAF7DA
:10826000E1FE2146BDE810400120FAF7DBBE000028
:108270009A9999999999A93F2DE9F04F8946002833
:1082800044D00A215A3090FBF1F00024C0EBC0002A
:10829000401CC6B24D464FF0800B4FF0080A17E065
:1082A000680700D100240BEB5400C4B20127AAEBED
:1082B000D508F019C1B208F0FF00FCF7FFFF00205D
:1082C00000F044F97F1CFFB2082FF2D36D1CEDB211
:1082D000182DE5D3002517E0680700D100240BEB2B
:1082E0005400C4B20127AAEBD508F019C1B208F0B6
:1082F000FF00FCF7E3FF204600F028F97F1CFFB2E7
:10830000082FF2D36D1CEDB24D45E5D3BDE8F08FDB
:108310000F490F4A91F82C1092F90C20042901D131
:10832000142A13DB002A01DA02290FD002F14601D8
:108330009D290BD20649002A91F8231002DD00F591
:10834000FA7001E0C0F5FA70FCF728BB7047000036
:10835000000000202DE9F041174E05462DED028B5F
:1083600000249FED148A4FF4B47700BF04EB44005F
:1083700000EBC4002844B84201DBA0F5B47000EE65
:10838000100AB8EEC00A20EE080A10EE100A01F03A
:108390001BF841EC100BFBF74FF951EC100B00F000
:1083A00051FA46F82400641C202CDFDBBDEC028B64
:1083B000BDE8F0814BFA8E3CE80200202DE9F04147
:1083C000174E05462DED028B00249FED148A4FF4C5
:1083D000B47700BF04EB440000EBC4002844B8426B
:1083E00001DBA0F5B47000EE100AB8EEC00A20EE72
:1083F000080A10EE100A00F0E7FF41EC100BFBF743
:1084000063FB51EC100B00F01DFA46F82400641CCD
:10841000202CDFDBBDEC028BBDE8F0814BFA8E3CFB
:10842000640200202DE9F04705462DED048B002461
:108430004FF4B4779FED1A9A1A4E084600F0D9FC13
:108440008946804604EB440000EBC4004219BA425E
:1084500001DBA2F5B47200EE102A49EC188BB8EEDD
:10846000C00A20EE090A10EE100A00F0ADFF41EC40
:10847000100BFBF729FB53EC182B51EC100B00F001
:10848000E3FC53EC182B00F00FFA00F085FC46F8E3
:108490002400641C202CD5DBBDEC048BBDE8F087E8
:1084A0004BFA8E3C740400202DE9F04100242DEDA0
:1084B000048B9FED169A164E00F09BFC0D46074666
:1084C00000EE104A45EC187BB8EEC00A20EE090A0F
:1084D00010EE100A00F078FF41EC100BFBF7F4FAF5
:1084E00053EC182B51EC100B00F0AEFC53EC182B96
:1084F00000F0DAF900F050FC46F82400641C202C4F
:10850000DEDBBDEC048BBDE8F0810000F90F493ED5
:10851000F80400200C494FF400428A624FF0904367
:108520009A62002210238B6203064FF0080301D5E4
:108530008B6100E08B6210238B614006521C000EA1
:10854000D2B2082AEED37047000400480C494FF419
:1085500000428A624FF090439A61002210238B629E
:1085600003064FF0080301D58B6100E08B621023F6
:108570008B614006521C000ED2B2082AEED370471F
:108580000004004810B52DED048BB0EE608AF0EECB
:10859000408A18EE100A00F017FF1B4C41EC190B33
:1085A000207E00EE100AF8EE400A88EE200A30EE37
:1085B000280A10EE100A00F007FF41EC100BB0EE95
:1085C000491AF0EE691AFAF737FF9FED101B51ECCC
:1085D000100B53EC112B00F037FC00F0ADFB94F8BE
:1085E0002C10072900D1093094F9001008445A30A2
:1085F0005A2803DD5A20BDEC048B10BD6FF05901E1
:108600008842F8DA0846F6E7000000200000006023
:1086100066A64C4010B510EE900A2DED048BB0EE1E
:10862000409A00F0D1FE41EC180B19EE100A00F050
:10863000CBFE41EC100BB0EE481AF0EE681AFAF7D8
:10864000FBFE9FED091B51EC100B53EC112B00F0BE
:10865000FBFB00F071FB064991F82C10072900D1B3
:108660000A30BDEC048B10BD0000006066A64C40D3
:10867000000000201749A1F180020B6C92F82D0038
:10868000001D03415BB29375896C014148B200F152
:108690001601D0752C291CD803F13F017E2918D86A
:1086A00092F90C10002908DB002800DA4042C1B220
:1086B000002B00DA5B4258B209E0002B01DD594281
:1086C0009175002800DA4042C1B292F91600FAF71B
:1086D000D9B870478000002010B5FCF7DFF907A17A
:1086E0000A48F7F7F7FD094A0A210320FCF7CEFAFA
:1086F000BDE810404FF4FA70FCF76AB920504C45C1
:108700004153452057414954000000003C020020DD
:108710002E4810B500F2291190F838208A7590F88B
:1087200036204A7080F8372090F824208A7090F81C
:108730003920CA7090F83A200A7190F82D304B71A8
:1087400090F82B208A7190F82C20CA7190F8302074
:108750000A7290F832204A7290F841208A72427F61
:10876000CA7290F844200A73827E4A7390F83E20C1
:108770008A7390F83320CA73B0F86C20140A4C74D2
:108780008A7400F18002012B546F1DD0C2F87C4026
:1087900032F8783F1C0ACC740B759288130A4B761A
:1087A0008A7610F82E2F4A7510F8132CCA75C278E5
:1087B0000A76428C130ACB760A77C28C130A4B775F
:1087C0008A778079C87710BD9467E1E700000020C0
:1087D0000A4910B501F22110CA7C42708A7CA0F1CE
:1087E000A10382701A89140AC47042719A89130A0B
:1087F0000371827191F82510C17110BD0000002035
:1088000010B500290AD00878002807D00548784418
:10881000F8F7F4FA002801D0002010BD024878448F
:1088200010BD00003A2800003228000081F000410D
:10883000704780F00040704721F00041704720F001
:108840000040704721F00042A2F16052B2F5801F53
:1088500001F0004328BFD2F17F6C0BD95FEA001C06
:1088600043EAC20242EB507018BF704728BF20F0A5
:1088700001007047B2F5801FBCBF184670474FEA31
:10888000410C1CF5001F02D2084600F013BE70B563
:1088900000F084FB00000089FFF7F6BF4FF00040B6
:1088A000A0F580007047000010B591EA030F48BFA3
:1088B00083F0004300F1A684841A71EB030C05D207
:1088C000121943EB0C03001B61EB0C01DFF824E1F0
:1088D0004FEA1154A4EB135C1EEA430F18BF9EEA43
:1088E000445F73D023EA0E03DCF1200E21EA045129
:1088F00043F4801332D322FA0CFE10EB0E0023FA5D
:108900000CFE41EB0E01CCF1200E03FA0EFE10EB33
:108910000E0051F10001B1F5801FCCF1200E32D2D2
:1089200001EB045112FA0EF2BDE8104058BF704737
:10893000401C38BF5FEA420218BF7047002814BFCE
:1089400020F0010041F100014FEA410313F5001F3F
:1089500038BF7047A1F1C04100F06EBB012A43EB64
:108960000302ACF1200CDCF11F0E32BF4FF0000E01
:1089700023FA0CF310EB030041EB0451B4EB115F4D
:10898000D0D0A1EB045101F5801149085FEA300015
:1089900001EB04510ED350F1000038BF12FA0EFE65
:1089A00008D1BDE81040C9E7401C38BF5FEA420269
:1089B000CAD1C3E7BDE810404FEA410313F5001FD9
:1089C00038BF7047A1F1C04100F036BB9EEA445F5A
:1089D00008D011EA5E0FBDE8104004BF01F000416D
:1089E00000207047BDE8104070B500F0D7FA00BF16
:1089F00064FBBE3E0000E0FF491058BFC1F140419A
:108A00005B1058BFC3F140438B42EFF300807047C7
:108A10002DE9C04130B4DFF8A0C23CEA111418BF00
:108A20003CEA131400F0EC8081EA03051CEA1114FF
:108A300044EAD57418BF1CEA131500F0C780A4EBF4
:108A400005044FF0004545EAC12145EAC32341EA48
:108A5000505143EA525304F17F74994204F50034B3
:108A60004FEAC0204FEAC22208BF904200F09C802B
:108A70004FEA13650FF24016765D4FEA134506FB89
:108A800005F7C7F1807706FB07F74FEAD737A7FB53
:108A900003687642C8F58038A7FB06CE38BFA8F138
:108AA000010807FB08E64FF0000EA6FB028CE6FB70
:108AB00003CEDCF1000CCEF1004E38BFAEF1010E5A
:108AC000A6FB0C584FF000074FF00005E6FB0E87A1
:108AD000A1FB08C6A0FB07CE16EB0E0645F100056C
:108AE000E1FB076515F1E04E7EBFA4F580345FEA37
:108AF00046066D4116F1800745F100054FEA17273C
:108B00004FEA066647EA0567A6F1DE46B6F1805FE2
:108B10004FEA15251FD9384624F0010C05EBC47126
:108B2000BCF1FE6F01EB0C1102D8F0BCBDE8008176
:108B300024425CBF01F5801E9EEAC47F02D4F0BCD3
:108B4000BDE80081244238D4F0BCA1F1C041BDE8A9
:108B5000004100F071BA4FEAD22242EA43524FEA92
:108B6000D323A7FB02864FEAD02040EA415007FBFF
:108B700003661EEA0E0F4FEAD12105FB026658BFBD
:108B8000A6EB0056B6EB00564FEA520E4EEAC37EF5
:108B900018EB0E0E56EB530EBDD518EB02085E41D6
:108BA0007F1C55F10005B6E74FF480154FF0000724
:108BB0004FF000064FF00008ADE7F0BC4FF00000AA
:108BC00001F1C04101F00041BDE8008111EA0C1F34
:108BD0000CEA131500D00CE013EA0C1F00F02580FE
:108BE0004FF00000F0BC81EA030101F00041BDE854
:108BF0000081F0BCBDE8004181EA030100F01CBA2D
:108C0000F0BCBDE8004170B500F0C8F9097EFC3E3B
:108C100000F007B881EA03014FF0000001F00041C5
:108C2000704781EA030100F007BAF0BCBDE80041DB
:108C30004FF0000021497047FFFDFBF9F7F5F4F212
:108C4000F0EEEDEBE9E8E6E4E3E1E0DEDDDBDAD8E7
:108C5000D7D5D4D3D1D0CFCDCCCBCAC8C7C6C5C445
:108C6000C2C1C0BFBEBDBCBBBAB9B8B7B6B5B4B35C
:108C7000B2B1B0AFAEADACABAAA9A8A8A7A6A5A447
:108C8000A3A3A2A1A09F9F9E9D9C9C9B9A9999980B
:108C90009797969595949393929191908F8F8E8EAE
:108CA0008D8C8C8B8B8A898988888787868585843B
:108CB00084838382828181800000FF070000F87F27
:108CC00051EA030C17D41CF5801F58BFBCF5801F58
:108CD00000F10680994218BF704708BF9042704764
:108CE00007D711F5801F58BF13F5801F19D499427B
:108CF0007047894270471CF5801F08D5BCF5801F5E
:108D0000F7D58B4218BF704708BF824270474FF4B7
:108D1000001C1CEB410F38BF1CEB430F01D28B42F0
:108D2000704770B500F03AF9922449004FF00051B5
:108D30004FF08053FFF760BE4FEA41034FEA5353B1
:108D4000A3F58063D3F11E03C8BFD3F1210C0CDD62
:108D50004FF0004242EAC12242EA505232FA03FC8A
:108D60008CEAE17CACEBE1707047102BC4BF0020B3
:108D7000704703F5787CBCF1FF3F04D06FF00042F0
:108D800082EA2100704770B500F008F9499224800A
:108D900000207047F2E700004FEA1153A3F580630B
:108DA000D3F11E03A8BFD3F1200C08DB4FF0004223
:108DB00042EAC12252EA505232FA03F070470942A5
:108DC0000BD4102BC4BF0020704703F5787CBCF196
:108DD000FF3F05D04FF0FF3070474FF00000704765
:108DE00070B500F0DBF800BF499224800020704786
:108DF000F0E710F0004248BF4042B0FA80F310FAAA
:108E000003F10AD0C3F11D0303F580634FEA41501B
:108E100002EB035202EBD12170474FF00000704784
:108E2000B0FA80F310FA03F10AD0C3F11D0303F581
:108E300080634FEA41504FEA035202EBD121704761
:108E40004FF0000070470000DFF848C170B51CEA21
:108E5000111E1EBF1CEA13159EEA0C0F95EA0C0F9B
:108E600000F06F8081EA030423EA4C134EEAD47EBB
:108E700021EA4C1141F4801143F48013AE44A1FB6C
:108E8000024CA0FB0365AEF17F7E361955EB0C0555
:108E9000A1FB034C4CF10003A0FB021C16EB0C06DB
:108EA000654153F10003094218BF46F0010613F46F
:108EB000007F0BD14FEA03314FEA0530340341EA1A
:108EC000155140EA16506FF003020AE04FEAC32141
:108ED0004FEAC520F40241EA555140EA56506FF07E
:108EE000020202EB2E4201EB025585EACE710AD056
:108EF0005FEA440C18BF24F0004450F1000041F137
:108F0000000120EAD47040F2FE7C624500D270BDC0
:108F1000A84214BF4FF080444FF04044002E08BFD9
:108F20000024BEF1806FA8BFA1F1C041BDE8704030
:108F300080F282804FF0000001F1C04101F0004159
:108F400070479EEA0C0F0CEA131518BF95EA0C0F38
:108F500006D04FF0000081EA030E0EF0004170BD14
:108F600000F01CF88900013E00F007B800F009B8D5
:108F70004FEA430C5FEA5C5C08D081EA030100F031
:108F80005BB84FEA410C5FEA5C5CF6D14FF0000041
:108F9000014970470000FF070000F87F0EF1020E44
:108FA0002EF0030E5EF8046B364205D4012A43EB23
:108FB000030515F5001F12D8012841EB010C1CF523
:108FC000001F0CD80ED14FEAD17C15F5001F0CEB19
:108FD0004C0C0CF1020C08BF4CEBD37C04E04FF0BE
:108FE000080C01E04FEAD37C0CEB4C0526FA05F6A1
:108FF00006F00706B6F1040C06D20EEB860CBDE8AF
:1090000070404CF0010C6047DFE80CF0090B0202E5
:109010004FF000414FF00000A1F5002170BD19464E
:109020001046012851EB010418BFD4F5001484BF89
:10903000002001F0004170BD0808A0F500114FEAC2
:109040003101704791EA030F10B581F000413FF5FF
:1090500033AC83F0004300F0D5B800002DE9F041B7
:1090600001F5801CBCF5001FC0F2A9804FEA115C1D
:1090700021EA0C510CF1FD0C41F480115FEA5C0C0B
:109080000CF5C07C01D34000494130A4890241EA7B
:10909000905187028E0E0A0CA45D04FB04F602FBBD
:1090A00006F6C6F14046A4FB0662F60D46EA4226E5
:1090B00006FB06F4A4FB01235242C3F1404338BF30
:1090C0005B1EA6FB02420024E6FB0324D20B42EA0D
:1090D0004446A6FB0623A1FB02E2A3FB07E4E3FB55
:1090E00061426442C2F1404E38BFAEF1010EA6FBB0
:1090F00004234FF00002E6FB0E32A2FB03463400CD
:10910000E2FB6264A1FB06E6A4FB07E8E4FB6168FE
:109110007642C8F1405838BFA8F10108A2FB06E426
:10912000A3FB08E5E2FB6854A1FB05E6A7FB04E806
:10913000E1FB648618F1200556F10006A809A8F1A4
:109140001B08B10908F03F08B8F10A0F40EA866031
:109150001CD901EB0C51BDE8F08100BFFCF5EEE835
:10916000E2DDD8D3CFCBC7C3C0BDB9B6B4B1AEACC6
:10917000A9A7A5A3A19F9D9B9A9896959392908F3E
:109180008D8C8B898887868584838281A0FB00688B
:1091900000FB01F208EB4208B8EB872807D534182A
:1091A00058EB0104D5D5401C51F10001D1E7341A28
:1091B00078EB0104CDD4401E71F10001C9E75FEAEC
:1091C0004C0C5FEA9C5C0DD105D34FF0000001F020
:1091D0000041BDE8F081BDE8F04170B5FFF7DEFE6B
:1091E0006DDBFFBEBDE8F0414FF000000049704765
:1091F0000000F87F10B591EA030F48BF83F00043E9
:109200003FF55AAB841A71EB030C07D212198CF09C
:10921000004C43EB0C03001B61EB0C01DFF8A4E1F5
:109220004FEA1154A4EB135C1EEA430F18BF9EEAE9
:10923000445F00F0B08023EA6E03524221EA0451F9
:10924000C3EB6E0338BF5B1EDCF1200E25D322FA80
:109250000CFE10EB0E0043FA0CFE41EB0E01CCF1BC
:10926000200E03FA0EFE10EB0E0051F10001CCF1BE
:10927000200E29D412FA0EF201EB0451BDE8104081
:1092800058BF7047401C1CBFB2F1004F7047002808
:109290000CBF491C20F00100704712EB020E43EB9B
:1092A000030218BF4FF0010E4EEA4202ACF1200C4F
:1092B000DCF11E0E54D943FA0CFE10EB0E0051F1F6
:1092C000FF31CCF11E0ED5D50EF1010E12FA0EFEB5
:1092D000404141EB010101EB445C5FEA5C5C10D969
:1092E00010EBDE7001EB045138BFBEF1004FBDE85A
:1092F000104018BF704700280CBF491C20F0010027
:10930000704730D24FEAD42C11F5001124F40064D8
:109310001BD0B1FA81F20B3AA41AA41ED2F1200399
:10932000914030FA03F31943904001EBCC71002CCB
:1093300001EB0451BDE81040A8BF704701F1C041E6
:109340004FF0000001F000417047B0FA80F310FACE
:1093500003F100D110BDE41A173C4805C90AE4E73F
:1093600001EB045110BD491001EB0451BDE8104060
:109370004FEA300002E04FF0000170474A0008BF9A
:109380000042F8D0B2F5001F28BF704701F000413D
:109390004FF0000070479EEA445F07D011EA5E0F6D
:1093A000BDE8104004BF002100207047BDE8104018
:1093B00070B5FFF7F3FD00BF40DFF63E83F00041DC
:1093C000104670470000E0FF43004FEAD30C4FEA1D
:1093D0003C0C43401FBF40070CF1605113F0FE4F9F
:1093E00070471CF0006F03D100200CF00041704763
:1093F0000CF0004343EA507010B540EACC0000F096
:109400000EF800BF000000924FEA0001FFF714BE03
:109410004FF000414FF00000A1F5002170470EF120
:10942000020E2EF0030E5EF8044B244204D44FEAE1
:109430004102B2F17F4F11D84FEA4003B3F17F4FA1
:109440000CD80ED14FEAD07CB2F17F4F0CEB4C0C14
:109450000CF1020C08BF4CEBD17C04E04FF0080C7F
:1094600001E04FEAD17C0CEB4C0324FA03F404F046
:109470000704B4F1040C06D20EEB840CBDE81040D6
:109480004CF0010C6047DFE80CF0070802024FF0D7
:109490000040A0F5800010BD0846420018BFD2F180
:1094A000807288BF00F0004010BD4FF04070E1EEC8
:1094B000100A7047FF2141EAD050C0057047F7F706
:1094C00000BA000000000404043C3C000008000056
:1094D000000800082CF4473B6C48B23B705BD83B5B
:1094E000395CA83B8EBA5F3BB25D47BB777ADFBC85
:1094F000F31C48BDBAF61FBD342CC5BDAC0B68BE0D
:10950000C1110D3E6CE40F3FC1110D3EAC0B68BEA6
:10951000342CC5BDBAF61FBDF31C48BD777ADFBC3D
:10952000B25D47BB8EBA5F3B395CA83B705BD83BF2
:109530006C48B23B2CF4473B67A029BD9C5775BDD6
:109540006FD1A5BD4AC9D4BDF8C102BEE1D3533F16
:10955000F8C102BE4AC9D4BD6FD1A5BD9C5775BD27
:1095600067A029BD84B46FBD5893B5BDDB14FCBDA5
:1095700017B123BE66BE5D3F17B123BEDB14FCBD31
:109580005893B5BD84B46FBD14BEA1BD6FEDFCBDD5
:10959000DC252FBEE9383F3FDC252FBE6FEDFCBD3B
:1095A00014BEA1BD5BC0FF3C45D0BF3D45D0BF3D13
:1095B0005BC0FF3C0000803FD417A5BFF8782A3F6E
:1095C000E66401BED315003FD315003F0000000044
:1095D000000000000000803F589B2E3A0000000071
:1095E000000000000000000000000000000000007B
:1095F000000000000000000000000000000000006B
:10960000000000000000000000000000000000005A
:10961000000000000000000000000000000000004A
:10962000000000000000000000000000000000003A
:10963000000000000000000000000000000000002A
:10964000000000000000000000000000000000001A
:109650000000000000000000000000000000C0E06A
:10966000F0F8FCFCFCFCFCFCFCFCFCFCFCFCF8F05A
:10967000E0C000000000FFFFFFFFFFFF0000000050
:1096800000000000FFFFFFFFFFFF00000000FFFFE2
:10969000FFFFFFFF0000000000000000FFFFFFFFD2
:1096A000FFFF00000000FFFFFFFFFFFF00000000C2
:1096B00000000000FFFFFFFFFFFF000000000307A6
:1096C0000F1F3F3F3F3F3F3F3F3F3F3F3F3F1F0F4A
:1096D000070300000000C0E0F0F8FCFCFCFCFCFC10
:1096E000FCFCFC0000000000000000000000000086
:1096F0000000000000FFFFFFFFFFFF000000000070
:1097000000000000000000000000000000FFFFFF5C
:10971000FFFFFF000000000000000000000000004C
:109720000000000000FFFFFFFFFFFF00000000003F
:10973000000000000000000000000000003F3F3F6C
:109740003F3F3F0000000000000000000000C0E0BC
:10975000F0F8FCFCFCFCFCFCFCFCFCFCFCFCF8F069
:10976000E0C0000000000000000000000000000059
:1097700000000000FFFFFFFFFFFF00000000C0E04F
:10978000F0F8FCFE7E7E7E7E7E7E7E7E7F3F1F0F1B
:10979000070300000000FFFFFFFFFFFF00000000C5
:1097A00000000000000000000000000000000307AF
:1097B0000F1F3F3F3F3F3F3F3F3F3F3F3F3F3E3C0D
:1097C0003830000000000C1C3C7CFCFCFCFCFCFC69
:1097D000FCFCFCFCFCFCF8F0E0C000000000000019
:1097E000000000000000000000000000FFFFFFFF7D
:1097F000FFFF00000000000000007E7E7E7E7E7E77
:109800007E7E7E7EFFFFFFFFE7C3000000000000BA
:10981000000000000000000000000000FFFFFFFF4C
:10982000FFFF0000000030383C3E3F3F3F3F3F3FDE
:109830003F3F3F3F3F3F1F0F070300000000FCFC7E
:10984000F8F0E0C00000000000000000C0E0F0F808
:10985000FCFC00000000FFFFFFFFFFFF0000000016
:1098600000000000FFFFFFFFFFFF00000000070FE8
:109870001F3F7F7F7E7E7E7E7E7E7E7EFFFFFFFFA0
:10988000FFFF0000000000000000000000000000DA
:1098900000000000FFFFFFFFFFFF000000000000CE
:1098A00000000000000000000000000003070F1F80
:1098B0003F3F00000000C0E0F0F8FCFCFCFCFCFCBA
:1098C000FCFCFCFCFCFC7C3C1C0C00000000FFFFD2
:1098D000FFFFFFFF0000000000000000000000008C
:1098E000000000000000070F1F3F7F7F7E7E7E7E0E
:1098F0007E7E7E7EFEFEFCF8F0E0000000000000B0
:10990000000000000000000000000000FFFFFFFF5B
:10991000FFFF0000000003070F1F3F3F3F3F3F3F97
:109920003F3F3F3F3F3F1F0F070300000000C0E0E5
:10993000F0F8FCFCFCFCFCFCFCFCFCFCFCFC7C3CB7
:109940001C0C00000000FFFFFFFFFFFF00000000F5
:109950000000000000000000000000000000FFFF09
:10996000FFFFFFFF7E7E7E7E7E7E7E7EFEFEFCF81B
:10997000F0E000000000FFFFFFFFFFFF000000001D
:1099800000000000FFFFFFFFFFFF000000000307D3
:109990000F1F3F3F3F3F3F3F3F3F3F3F3F3F1F0F77
:1099A0000703000000000C1C3C7CFCFCFCFCFCFCE5
:1099B000FCFCFCFCFCFCF8F0E0C000000000000037
:1099C000000000000000000000000000FFFFFFFF9B
:1099D000FFFF000000000000000000000000000089
:1099E00000000000FFFFFFFFFFFF0000000000007D
:1099F000000000000000000000000000FFFFFFFF6B
:109A0000FFFF000000000000000000000000000058
:109A10000000000003070F1F3F3F00000000C0E0F0
:109A2000F0F8FCFCFCFCFCFCFCFCFCFCFCFCF8F096
:109A3000E0C000000000FFFFFFFFFFFF000000008C
:109A400000000000FFFFFFFFFFFF00000000C3E772
:109A5000FFFFFFFF7E7E7E7E7E7E7E7EFFFFFFFF1E
:109A6000E7C300000000FFFFFFFFFFFF0000000052
:109A700000000000FFFFFFFFFFFF000000000307E2
:109A80000F1F3F3F3F3F3F3F3F3F3F3F3F3F1F0F86
:109A9000070300000000C0E0F0F8FCFCFCFCFCFC4C
:109AA000FCFCFCFCFCFCF8F0E0C000000000FFFF48
:109AB000FFFFFFFF0000000000000000FFFFFFFFAE
:109AC000FFFF00000000070F1F3F7F7F7E7E7E7E2E
:109AD0007E7E7E7EFFFFFFFFFFFF00000000000094
:109AE000000000000000000000000000FFFFFFFF7A
:109AF000FFFF0000000030383C3E3F3F3F3F3F3F0C
:109B00003F3F3F3F3F3F1F0F0703000000000000A3
:109B10000000000000000000000000000000000045
:109B20000000000000000000000000000000000035
:109B30000000000000000000000000000000000025
:109B40000000000000000000000000000000000015
:109B50000000000000000000000000000000000005
:109B600000000000000000000000000000000000F5
:109B700000000000000000000000000000000000E5
:109B800000000000000000000000000000000000D5
:109B900000000000000000000000000000000000C5
:109BA00000000000000000000000000000000000B5
:109BB00000000000000000000000000000000000A5
:109BC0000000000000000000000000000000000095
:109BD0000000000000000000000000000000000085
:109BE0000000000000000000000000000000000075
:109BF0000000000000000000000000000000000065
:109C00000000000000000000000000000000000054
:109C10000000000000000000000000000000000044
:109C20000000000000000000000000000000000034
:109C30000000000000000000000000000000000024
:109C40000000000000000000000000000000000014
:109C50000000000000000000000000000000000004
:109C600000000000000000000000000000000000F4
:109C700000000000000000000000000000000000E4
:109C800000000000000038FCFC3800000000000D5F
:109C90000D000000000E1E00001E0E00000000005F
:109CA0000000000020F8F820F8F82000020F0F0252
:109CB0000F0F0200387C444747CC9800060C083848
:109CC000380F070030300080C06030000C06030100
:109CD000000C0C0080D87CE4BCD84000070F0808BA
:109CE000070F080000101E0E00000000000000001A
:109CF000000000000000F0F80C0400000000030762
:109D00000C0800000000040CF8F000000000080C33
:109D10000703000080A0E0C0C0E0A08000020301B3
:109D200001030200008080E0E0808000000000036A
:109D30000300000000000000000000000000101EF2
:109D40000E00000080808080808080000000000085
:109D50000000000000000000000000000000000CF7
:109D60000C00000000000080C06030000C06030101
:109D700000000000F8F80CC40CF8F00003070C0811
:109D80000C070300001018FCFC0000000008080F7E
:109D90000F080800080C84C4643C18000E0F090862
:109DA000080C0C00080C444444FCB800040C0808DF
:109DB000080F0700C0E0B098FCFC8000000000081D
:109DC0000F0F08007C7C444444C48400040C080841
:109DD000080F0700F0F84C4444C08000070F080843
:109DE000080F07000C0C0484C47C3C0000000F0F1B
:109DF00000000000B8FC444444FCB800070F080809
:109E0000080F0700387C444444FCF80000080808A8
:109E10000C070300000000303000000000000006C6
:109E20000600000000000030300000000000080EB6
:109E3000060000000080C060301808000000010328
:109E4000060C080000202020202020000001010135
:109E5000010101000008183060C0800000080C06F5
:109E600003010000181C04C4E43C18000000000DAD
:109E70000D000000F0F008C8C8F8F000070F080B4C
:109E80000B0B0100E0F0988C98F0E0000F0F000041
:109E9000000F0F0004FCFC4444FCB800080F0F083E
:109EA000080F0700F0F80C04040C180003070C0856
:109EB000080C060004FCFC040CF8F000080F0F0866
:109EC0000C07030004FCFC44E40C1C00080F0F0802
:109ED000080C0E0004FCFC44E40C1C00080F0F08E6
:109EE00000000000F0F80C84848C980003070C0834
:109EF00008070F00FCFC404040FCFC000F0F000076
:109F0000000F0F00000004FCFC0400000000080F1C
:109F10000F08000000000004FCFC0400070F080804
:109F20000F07000004FCFCC0E03C1C00080F0F0001
:109F3000010F0E0004FCFC0400000000080F0F08D5
:109F4000080C0E00FCFC387038FCFC000F0F000001
:109F5000000F0F00FCFC3870E0FCFC000F0F00004D
:109F6000000F0F00F8FC040404FCF800070F0808B9
:109F7000080F070004FCFC44447C3800080F0F085D
:109F800000000000F8FC040404FCF800070F080EB1
:109F90003C3F270004FCFC44C4FC3800080F0F00C1
:109FA000000F0F00183C6444C49C1800060E0808FB
:109FB000080F0700001C0CFCFC0C1C000000080F24
:109FC0000F080000FCFC000000FCFC00070F080864
:109FD000080F0700FCFC000000FCFC000103060C5D
:109FE00006030100FCFC000000FCFC00070F0E0350
:109FF0000E0F07000C3CF0E0F03C0C000C0F0301CE
:10A00000030F0C00000C7CC0C07C3C000000080F5B
:10A010000F0800001C0C84C4643C1C000E0F0908CF
:10A02000080C0E000000FCFC0404000000000F0FF0
:10A03000080800003870E0C0800000000000000147
:10A0400003070E0000000404FCFC000000000808E8
:10A050000F0F0000080C0603060C080000000000AB
:10A060000000000000000000000000002020202070
:10A070002020202000000307040000000000000052
:10A080000000000000A0A0A0E0C00000070F08082A
:10A09000070F080004FCFC2060C08000000F0F08C0
:10A0A000080F0700C0E0202020604000070F0808CC
:10A0B000080C040080C06024FCFC0000070F0808A6
:10A0C000070F0800C0E0A0A0A0E0C000070F08082C
:10A0D000080C040040F8FC440C180000080F0F089E
:10A0E00000000000C0E02020C0E02000276F4848AA
:10A0F0007F3F000004FCFC4020E0C000080F0F0080
:10A10000000F0F00000020ECEC0000000000080F22
:10A110000F0800000000000020ECEC000030704050
:10A12000407F3F0004FCFC80C0602000080F0F014E
:10A13000030E0C00000004FCFC0000000000080FEF
:10A140000F080000E0E060C060E0C0000F0F0007F3
:10A15000000F0F0020E0C02020E0C000000F0F0023
:10A16000000F0F00C0E0202020E0C000070F08080B
:10A17000080F070020E0C02020E0C000407F7F489B
:10A18000080F0700C0E02020C0E02000070F0848AB
:10A190007F7F400020E0C06020E0C000080F0F0873
:10A1A0000000000040E0A02020604000040C0909ED
:10A1B0000B0E04002020F8FC202000000000070FF8
:10A1C000080C0400E0E00000E0E00000070F0808D1
:10A1D000070F080000E0E00000E0E0000003070CCB
:10A1E0000C070300E0E0008000E0E000070F0C0730
:10A1F0000C0F07002060C080C0602000080C07031F
:10A20000070C0800E0E0000000E0E000474F48488D
:10A21000683F1F00606020A0E06020000C0E0B096A
:10A22000080C0C00004040F8BC04040000000007CB
:10A230000F080800000000BCBC0000000000000F78
:10A240000F000000000404BCF84040000008080FA4
:10A2500007000000080C040C080C040000000000BB
:10A2600000000000E0F0988C98F0E0000F0F000074
:10A27000000F0F0004FCFC4444CC8C00080F0F08B6
:10A28000080F070004FCFC4444FCB800080F0F084A
:10A29000080F070004FCFC04040C0C00080F0F0856
:10A2A0000000000000F8FC0CFCF800001C0F0F0878
:10A2B0000F0F1C0004FCFC44E40C1C00080F0F08EA
:10A2C000080C0E000C3CE0FCE03C0C000C0F010FF5
:10A2D000010F0C00080C444444FCB800040C0808AE
:10A2E000080F0700FCFC80C060FCFC000F0F0100A1
:10A2F000000F0F00FCFC80C260FCFC000F0F01008F
:10A30000000F0F0004FCFCC0E03C1C00080F0F0015
:10A31000010F0E0000F0F81C0CFCFC00080F0F00F1
:10A32000000F0F00FCFC387038FCFC000F0F000021
:10A33000000F0F00FCFC404040FCFC000F0F000031
:10A34000000F0F00F8FC040404FCF800070F0808D5
:10A35000080F0700FCFC040404FCFC000F0F0000C5
:10A36000000F0F0004FCFC44447C3800080F0F0869
:10A3700000000000F0F80C04040C180003070C089F
:10A38000080C0600001C0CFCFC0C1C000000080F54
:10A390000F0800001C3C60C080FCFC0000000C0D9D
:10A3A00007030100F0F808FC08F8F0000103020FB1
:10A3B000020301000C3CF0E0F03C0C000C0F030128
:10A3C000030F0C00FCFC0000FCFC00000F0F080851
:10A3D0000F1F1800387CC08080FCFC0000000000CB
:10A3E000000F0F00FC00FCFC00FC00000F080F0F2A
:10A3F000080F0000FC00FCFC00FC00000F080F0F21
:10A40000081F180004FCFC4040C0C000080F0F08E3
:10A41000080C0F00FCFC40C0C000FC000F0F080C33
:10A420000F000F0000FCFC4040C0C000000F0F08F0
:10A43000080C0F000C0404C4CCF8F0000C08080849
:10A440000C070300FCFC80F80404F8000F0F000761
:10A45000080807000078CC8484FCFC00080C060384
:10A46000010F0F0000A0A0A0E0C00000070F080827
:10A47000070F0800E0E02020202000000F0F09094E
:10A4800009060000E0E0A0A0A04000000F0F0808AF
:10A4900008070000E0E02020206000000F0F00000F
:10A4A0000000000000E02020E00000001C0F0C0C69
:10A4B0000F1C0000C0E0A0A0A0E0C000070F08082B
:10A4C000080C040020E080E080E02000080F010F6D
:10A4D000010F0800402020A0E060000004080909E6
:10A4E00006060000E0E0000080E000000F0F02011F
:10A4F000000F0000E0E0001080E000000F0F0201FC
:10A50000000F000004FCFC80C0602000080F0F0159
:10A51000030E0C0000E02020E0E00000080700002F
:10A520000F0F0000E0C00000C0E000000F000101BC
:10A53000000F0000E0E00000E0E000000F0F01016C
:10A540000F0F0000C0E0202020E0C000070F080827
:10A55000080F0700E0E02020E0E000000F0F0000FF
:10A560000F0F000020E0C02020E0C000407F7F48A7
:10A57000080F0700C0E0202020604000070F0808F7
:10A58000080C04002020E0E02020000000000F0F55
:10A590000000000060C08000E0E000000C0C070339
:10A5A00001000000C020F0F020C0000003040F0FE5
:10A5B000040300002060C080C0602000080C070376
:10A5C000070C0800E0E0000000E000000F0F0808A2
:10A5D000080F1800E0E00000E0E0000001030202C4
:10A5E0000F0F0000E000E0E000E000000F080F0F98
:10A5F000080F0000E000E0E000E000000F080F0F8F
:10A60000081F100000000000000000000000000013
:10A6100000000000E080800000E000000F08080754
:10A62000000F00008080808080808000000000009B
:10A630000000000040202020E0C0000004080809BD
:10A640000F070000E000C02020C000000F01070835
:10A6500008070000C0202020E0E0000008050301FA
:10A660000F0F0000000000000000000000000000CC
:10A6700000000000000000000000002F00000007A4
:10A68000000700147F147F14242A7F2A1223130842
:10A69000646236495522500005030000001C224127
:10A6A000000041221C0014083E081408083E080857
:10A6B0000000A06000080808080800606000002092
:10A6C000100804023E5149453E00427F400042616D
:10A6D0005149462141454B311814127F10274545F9
:10A6E00045393C4A49493001710905033649494910
:10A6F00036064949291E003636000000563600004D
:10A7000008142241001414141414004122140802E5
:10A7100001510906324959513E7C1211127C7F4980
:10A720004949363E414141227F4141221C7F4949EE
:10A7300049417F090909013E4149497A7F080808D2
:10A740007F00417F41002040413F017F08142241AA
:10A750007F404040407F020C027F7F0408107F3E14
:10A760004141413E7F090909063E4151215E7F0971
:10A77000192946464949493101017F01013F4040BD
:10A78000403F1F2040201F3F4038403F63140814C3
:10A790006307087008076151494543007F41410044
:10A7A00001060830400041417F00040201020440DC
:10A7B00040404040000305000020545454787F4836
:10A7C0004444383844444420384444487F3854543E
:10A7D0005418087E09010218A4A4A47C7F0804046C
:10A7E0007800447D40004080847D007F1028440034
:10A7F00000417F40007C041804787C080404783809
:10A8000044444438FC2424241818242418FC7C08CC
:10A810000404084854545420043F4440203C404021
:10A82000207C1C2040201C3C4030403C4428102808
:10A83000441CA0A0A07C4464544C4400107C8200C2
:10A840000000FF000000827C100008040810087C53
:10A850001211127C7F494949317F4545453A7F01B4
:10A86000010103603F213F607F49494941730C7FEB
:10A870000C732141494D337F1008047F7E2011085D
:10A880007E7F08142241403F01017F7F0608067F3A
:10A890007F0808087F3E4141413E7F0101017F7FE3
:10A8A000090909063E4141412203017F0103612656
:10A8B0001806011C227F221C63140814633F202009
:10A8C0003F60070808087F7F407F407F3F203F2090
:10A8D0007F017F4848307F4878007F7F48483000BC
:10A8E0004149492A1C7F103E413E661909097F20D3
:10A8F000545478403E494545387E4A4A34007C04E9
:10A90000040C00384545493E38545454184C307CAA
:10A91000304C24424A34007C20107C007C21117C85
:10A92000007C10284400403C04047C7C0810087C17
:10A930007C10107C0038444444387C04047C00FCC7
:10A9400018242418384444442804047C04044C90FB
:10A9500090907C18247E241844281028443C202001
:10A960003C601C10107C007C407C407C3C203C20E7
:10A970007C047C5070007C5070007C7C5070000027
:10A98000424252523C7C10384438402C127E000027
:10A990000000000030313233343536373839414227
:10A9A0004344454640305800303132333435363731
:10A9B00038396162636465664030780004000008DD
:10A9C0000000000000000002000100001000000074
:10A9D00004FA97999999D93FAF788E1DC571CC3FEC
:10A9E0009FC678D0099AC33F935555555555E53FB5
:10A9F000599322942449D23FDE03CB966446C73F45
:10AA000044523EDF12F1C23F4FBB610567ACDD3FF0
:10AA1000182D4454FB21E93F9BF681D20B73EF3F85
:10AA2000182D4454FB21F93FE2652F227F2B7A3CFD
:10AA3000075C143326A6813CBDCBF07A8807703CB6
:10AA4000075C143326A6913CC4EB98999999C9BF29
:10AA5000711623FEC671BCBF6D9A74AFF2B0B3BF5E
:10AA60009AFDDE522DDEADBF2F6C6A2C44B4A2BF1E
:10AA70000D5555555555D53FFF8300922449C23F8A
:10AA80006E204CC5CD45B73F513DD0A0660DB13FBE
:10AA9000EB0D76244B7BA93F11DA22E33AAD903FD0
:10AAA0004C5555555555A53F7751C1166CC156BFEC
:10AAB0009015CB19A001FA3EAD529C804F7E92BEFC
:10AAC000C4B1B4BD9EEE213ED43888BEE9FAA8BD1B
:10AAD000000000000000000000004054FB21F93F8E
:10AAE0003163621A61B4D03D0000601A61B4D03D98
:10AAF0007370032E8A19A33B0000002E8A19A33B12
:10AB0000C14920259A837B39000000000000000025
:10AB10006E83F9A22915444ED15727FCC0DD34F5C8
:10AB2000999562DB4190433CAB6351FE61C5BBDE4E
:10AB30003A6E24B7E0D24D42EA2E49061C92D10962
:10AB40001CEB1DFE3EA729B1F53582E88444BB2EDF
:10AB500026709CE9417E5FB439D69139F43953832C
:10AB60008B5F849C3B28F9BDFF97F81F0F9805DE8B
:10AB70008B112FEF1F6D0A5ACF7E366DB709CB2789
:10AB8000663F464F2DEA5F9EC7BA27757BF1E5EB1E
:10AB9000F739073DEA92528AB15FFB6B085D8D1F62
:10ABA000A6F810111111813FD561C119A0012ABF6A
:10ABB0007DFEB157E31DC73EEB9C2B8AE6E55ABEEE
:10ABC0007CD5CF5A3AD9E53D7AFE10111111C13F1B
:10ABD00037D60684F464963F280356C9226D6D3F2C
:10ABE0000165F2F2D844433FA69237A0887E143F15
:10ABF000735360DBCB75F3BEFE41B31BBAA1AB3F11
:10AC000093846EE9E326823F1583E0FEC8DB573F5D
:10AC100068108D1AF726303FE9A7F0320FB8123FBF
:10AC2000D47ABF74702AFB3E02400000000000A0EE
:10AC30000000000005400000000000C80000000007
:10AC40000C4000000000409C000000001940000083
:10AC50000020BCBE0000000034400000BFC91B8EB5
:10AC600000000004B5400000504BCFD06607E2CF93
:10AC7000010000006C4100003E8251AADFEEA734C3
:10AC800001000000D9420000DCB5A0E23A301F9775
:10AC9000FFFFFFFFB4450000FD25A0C8E9A3C14F99
:10ACA000FFFFFFFFFF3F00000000008000000000EA
:10ACB000FF3F00000000008000000000564F4C2EB7
:10ACC0004645202020202000412F4D20464153544E
:10ACD000202020202000000053454E5320464520D0
:10ACE00020202000564F4C2E554D4520202020007E
:10ACF000444953504C4559202020200020204245F3
:10AD0000414348202020000020205041524B202069
:10AD100020000000412F4D20534C4F572020200091
:10AD2000564F4C2E544F4E4520200000484F542083
:10AD300053544F4E4520200046494C544552204C18
:10AD400050202000504F5745522020004C454420B1
:10AD500042524947485420200000000057524954AD
:10AD6000452020202D206F72202B20004449534382
:10AD70002D200000564F4C2E572E5349472E2000B1
:10AD8000564F4C2E534348454D45200020525542C6
:10AD90004249534820000000412F4D204D45444971
:10ADA000554D20002043752B41672B202A000000C1
:10ADB0005752495445202D206F72202B000000006F
:10ADC000465245512E000000D093D1802ED0A1D004
:10ADD000BB2ED0A1D0B8D0B32E00000030000000B0
:10ADE00050524F46494C4500464552524954450041
:10ADF0004742562F474246005059432F454E470081
:10AE00002053656142454143480000004741494E97
:10AE1000000000004241545445525900D09CD09546
:10AE2000D094D0ACD18AD0BFD0BBD18ED18100001C
:10AE3000D0ADD09AD0A0D090D09DD18AD18AD18ADD
:10AE4000D18AD18A00000000D0A4D098D09BD0AC89
:10AE5000D0A2D0A0D18AD18AD18AD18AD18A000049
:10AE6000D18AD18AD18AD09FD09ED09BD095D18AC9
:10AE7000D18AD18AD18A0000D0AFD0A0D09AD09EFA
:10AE8000D0A1D0A2D0ACD18AD18AD18AD18A0000F7
:10AE9000D0A2D09ED09DD18AD097D092D0A3D09A64
:10AEA000D090D18AD18AD18A00000000D18AD18A7B
:10AEB000D18AD09FD09BD0AFD096D18AD18AD18A67
:10AEC00000000000D0A2D09ED09AD18AD18AD18A27
:10AED00000000000D18AD18AD18AD09FD090D0A022
:10AEE000D09AD18AD18AD18A00000000D093D09E16
:10AEF000D0A0D18AD09AD090D09CD09DD098D18A21
:10AF0000D18A0000D0A7D0A3D092D0A1D0A2D18A5C
:10AF1000D096D095D09BD18AD18A0000D18AD18A8F
:10AF2000D18AD09CD0A3D0A1D09ED0A0D18AD18AE2
:10AF300000000000D093D0A0D09ED09CD09AD09E8C
:10AF4000D0A1D0A2D0ACD18AD18A0000D09CD09E12
:10AF5000D0A0D0A1D09AD18AD09FD09BD0AFD0968C
:10AF6000D18A0000D090D0A2D090D09AD090D18A2F
:10AF7000D093D0A0D09ED09CD18A0000D091D09008
:10AF8000D09BD090D09DD0A1D18A0000D094D098F1
:10AF9000D0A1D09AD18C0000D0A7D0A3D09220D03D
:10AFA00096D095D09BD095D097D09000D091D09549
:10AFB000D097D18AD096D095D09BD095D097D0906D
:10AFC00000000000D0A7D090D0A1D0A2D09ED0A2E7
:10AFD000D0900000D0A4D095D0A0D0A0D098D0A27E
:10AFE00000000000D0A7D090D0A1D0A200000000A7
:10AFF000D092D0A1D095D18AD09CD095D0A2D0901B
:10B00000D09BD0AB00000000D09FD0A0D09ED0A499
:10B01000D098D09BD0AC0000D091D090D0A2D0904E
:10B02000D0A0D095D0AF000064B000080000002090
:10B030003C020000C401000854B100083C0200209A
:10B040005C110000200200081C000000430000000A
:10B05000F8FFFFFF0C0000000E0000000F000000D2
:10B060002E00000032A6620159070136C5BB99BD0A
:10B0700046C5BC7493BC0A3B2C5E01768701020472
:10B080000A5A13170A01020801081501050157178A
:10B0900064015001012B14B414019303B413E0AD07
:10B0A000140808B0140814AE1B0818081A0C08136A
:10B0B000C4AF1B08C0181AE4081AE8081AD4081A02
:10B0C000B0081A7C081AF0082AF81C12AC1B0834C5
:10B0D000101A800C1A64081A74081AC8041ABC18CA
:10B0E0001A04101A200C1A904C1A44081AC4081A90
:10B0F00038081A48081A6C081A8C201A4C081A7852
:10B10000101AF0301A30081A2C101AEC081AD8103D
:10B110001A98201A5C101ADC041A14041AF0101A77
:10B1200098081AAC081AC8201A60281AFC081AAC29
:10B13000081119041A4C181A8C201A1C082A08B075
:10B1400019142AA410292023127A400880C0E0F0A4
:04B15000F8FCFE0009
:040000050800018965
:00000001FF
